:100000000C9496080C94C3080C94C3080C94C30871
:100010000C94C3080C94C3080C94C3080C94C30834
:100020000C94C3080C94C3080C94C3080C94C30824
:100030000C94053A0C94C3080C94C3080C94C308A0
:100040000C94C3080C943C250C94C3080C94C3086E
:100050000C94C3080C94C3080C94C3080C94C308F4
:100060000C94C3080C94DC390C94B2390C94C3087A
:100070000C94C3080C94C3080C94C3080C94C308D4
:100080000C94C3080C94C3080C94C3080C94C308C4
:100090000C94C3080C94C3080C94C3080C94C308B4
:1000A0000C94C3080C94C3080C94C3080C94C308A4
:1000B0000C94C3080C94C3080C94C3080C94C30894
:1000C0000C94C3080C94C3080C94C3080C94C30884
:1000D0000C94C3080C94C3080C94C3080C94C30874
:1000E0000C94C3080C948B1E0C944F140C94F23790
:1000F0000C9482140C949D2E0C9413350C940824AB
:100100000C94FD370C94A21A0C94872F0C94FC14B9
:100110000C94882C0C94DC2A0C94F7200C94502A14
:100120000C941C2C0C941B2E0C9462240C943135D2
:100130000C94231E0C944E390C94A6390C94201F59
:100140000C94D3110C945A140C94D5330C948F2D19
:100150000C941C1D0C94D4210C943C190C94F8188C
:100160000C9417200C94B8100C9412110C94791460
:100170000C946E130C94EF210C9413190C948F268D
:100180000C94991D0C947B340C94D31F0C94183050
:100190000C9410280C94C41E0C942E1C0C94D6267F
:1001A0000C9478230C944B230C94DD330C9435126F
:1001B0000C94E6300C94332B0C942E110C94712B70
:1001C0000C94121C0C944B390C9411350C943C2853
:1001D0000C9481110C94C2220C94731A0C946D2A05
:1001E0000C94832C0C94D6130C94831F0C947616C9
:1001F0000C940B2B0C94B8240C94581B0C941417CF
:100200000C94F3380C94CF230C94F3260C9493396C
:100210000C94A62F0C941F2A0C94D5260C94BC2E5B
:100220000C94A5330C9482280C9405230C94722012
:100230000C94841B0C94C9160C943A220C94C5217E
:100240000C9439230C943A240C94462C0C94EA24F4
:100250000C94DA160C9432150C94C1340C94FA20D8
:100260000C94FB120C94631A0C94A2110C948C1332
:100270000C94FB270C94F61B0400040000040700F8
:100280000400020000040000000000000004000060
:10029000000004040404000407040400000000003B
:1002A0000407070400000400020204040004040020
:1002B0000404040400000404040002030000020417
:1002C000000002020004000004000404040400040E
:1002D000040004000004000400000000000000000E
:1002E00001020102D6023C28020100018510B8106B
:1002F00003010001D5023923040400044E10B82480
:10030000050200025210841B060001000000822832
:1003100007020002D602832C0802000252108B1E34
:1003200009010001D50205230A030003D202351298
:100330000B020002D0024B230C030003CD02A533B5
:100340000D00010000004E390E080008C502782398
:100350000F060006BF02FC14100200025210DC2A35
:10036000110201018010FB2712030003BC02791463
:1003700013040004B8028F2D14010001D5021211DC
:1003800015050005B302201F16030003B002CF239A
:100390001704000354103C1918050005AB028C1318
:1003A00019010001D502332B1A0300027110872FA7
:1003B0001B080008A302C1341C0300027110FD37A2
:1003C0001D030002711018301E020002D0020B2B18
:1003D0001F050003A002FA202002000252105A1446
:1003E000210300027110F61B220400047A10581B2E
:1003F000230400046D10082424030003B002131921
:10040000250300027110731A260300027110C91629
:10041000270001000000A639280600069A02A62F30
:100420002900010000004B392A010001D502712B7F
:100430002B0400044E10DD332C030003CD02EA240C
:100440002D000100000093392E0400039702231EA3
:100450002F0500059202882C300400046D10F3383B
:1004600031020002D0026E1332030103D202D626FB
:100470003303000373108214340300027110121C42
:10048000350600069A0232153602000252109D2EE1
:100490003704000363101C2C38020102D00210281C
:1004A000390500058D0214173A020002D0027B3490
:1004B0003B010001D502D3113C010001D502D53327
:1004C0003D030003D202E6303E08000885022E1CE0
:1004D0003F0500058002462C400300027110631A9C
:1004E00041030003B002A211420400037D0276160C
:1004F000430200025210C22244010001D502BC2E68
:100500004500010000002E11460200025210502A40
:10051000470500057802C41E480200025210FB1273
:1005200049030003D202D6134A0400044E10DA161F
:100530004B0001000000D5264C000500000078DAD1
:10054000A519696FDBC8F5AF700504ED16B621512A
:100550002225B9C8075FD9A61B27DE386E0A140505
:1005600041932369605ECB217D74E1FFDE77CC454A
:100570004AC92EDA00816638EF9879F77BFE6D72F2
:10058000DFCB224F1E45AB645DA9C9E9649B65A71B
:10059000C19F7FBAB8F831884E1627D3E05E567DEA
:1005A000270B855F3FDE05E77AFB63109E84F149E8
:1005B000389DC5D359184D8E26595D96699503917E
:1005C000DF266951D459DA89A496B90AB2BAAFBA0A
:1005D000B76FB2C969383D02965D07BC92347B089B
:1005E000E018BE7B002BEF3CCFCD79532BFA91D591
:1005F000DB377DD0F44591F40DC1CF170EE1D75E06
:10060000B42F96245CE001A15BA1BAA493D983E244
:100610005DD7A6952A659718A681ACE0FDFA7E33D2
:10062000784721D23651BBBECBEBA76A721AE3D30F
:10063000AA8DDCC28D9E8BF922322C5423135EC20C
:100640003D420755A545BD4D64656F4FD79E9C46FD
:100650002B0BA3AF6C20789B3831441692BE897661
:10066000486B2082C5C202E7722BBBB448EABE1BAE
:10067000213CA6452F709F8B4DDA175D623F94E9B0
:100680007392F76DDA8101D03543474F803ABBBA98
:1006900019D0CA06CC43F7EE5DBE582C575303DC85
:1006A000AA44F31666912FEC2AB2ABD8AE96762503
:1006B0008AF4C5EA0C34E098C830330C60097264DF
:1006C000AD82A9E12F980CA89B9196EE1965D3AF46
:1006D000C368EA231ABD450EAA1275239F453192BD
:1006E0005C9E7669A2E47F80C1AE076FE8129498A1
:1006F00067504AC02759F9F79D5BA2CD5379401B3B
:10070000D90B1899A3A175B1EBC7DA812F7BEA99B0
:1007100039DB00031C1346B7EAE4A3487672BBA397
:1007200017CE421F1EAC735B887D0B0EEC59D2BDF9
:10073000348230E30127EB118790F55152AAEDDBAB
:10074000377F811010CE07B84FB2DB811892CC985A
:100750003C509F3A886EB90EAD7A326B382A2B1E08
:10076000EC5AE676F95265C9D04682ACCC93B1D941
:100770002C7C0EA2699C17E136D1D69CCBD62C39A5
:100780001010B083EA0B257CA24B4BB4DB89B6ACCE
:10079000C1419B8312F58F9D50E72E9C7465D6A7AF
:1007A000ADB58DF639D9F3EEA0B31FD1F23A590A9F
:1007B00036EE99A3D2A23CAC5841EEB9B8EFC19C39
:1007C000EB06E022B3052A5BB265D6CF6C690E5A00
:1007D00091429C6D73D1223FF4200E56B101786A8C
:1007E0006527F620D0681910A42C4AD16E4595BD16
:1007F00024182E4048703D1D3B925D5D8ABDA0AC23
:10080000D2B2F13D40EF6D481E066DB8BB8B57FC70
:100810005E2BE4566EB7A2C55728741034F8856372
:100820004E29012E9576C24A687D34D94888D1E098
:10083000D209CB30C8DA8C43DFD1640BDE4CD784CD
:1008400057447A4B4060B16BDEF70DEA011881AC7A
:1008500075D04B14704CC0086D48C7358B3A0A47A9
:1008600060A80503E63432076A1899CA3A979B973D
:1008700004D46D69B582BC2AD09909AE80A71A6DDF
:10088000C668ACC6213C7E4B0AC171238E1950ABA1
:10089000738F3D2427998BAA03E641BDD90017F237
:1008A0002B9B92808F8990F40C2BCF45E89DF44DC3
:1008B000EE64CD797BD77B6C2290292B65944C0F0D
:1008C000E76B603B1D2190367B1747A2B5051827C3
:1008D000DEFFD1DC4A676E3A00BB1D140F5B40DCC3
:1008E00089ECC14BD7E1D2DC6194AEED0D9A1A5C74
:1008F0007ACCDF8B2A067F94AABE259578364218DB
:100900004B255E1980BDA0FF8DCA086D1A62BCDC44
:10091000F0931696C0A130F70D1A9EE40682C330FC
:10092000C122EAC5A122C592ABFD34BA9C1B9451E9
:1009300016B5E0562F407F6680316CDB548FCAE0DD
:1009400048654C79476502FC4A302EB01D4AE0608C
:10095000FF6649F81C02C6FC000AAC1161FC378C2A
:100960002A2CB8F71E0C3D8092BE2539A80040DC29
:100970006B46AAC4B3BE01E425EBA5B265C29ABB1F
:1009800011C7EF5413F03E50A297D8B1F2DD38E30F
:10099000745E196A38CFAFBDD378614E3B2CB8FC7A
:1009A00054A7EB2F8859C2ABC3E0397387A2EA4D35
:1009B000F794B6C2C72DA5AA4D622B6B250F65FC17
:1009C0003DA29126FAED77CC51F4544C7C2F208730
:1009D000EB21D4E1781CC60845654382511F62991A
:1009E000C422CCBA581839004A3668BC9C8E029B87
:1009F0009DBC5C05EA00923AE90F444D21D9466C52
:100A0000763F04656C94213AE7010700923307D7DB
:100A1000F9C58468EA566732F653DA5B2311CF8D45
:100A200004957869731E594AA35778403108984352
:100A3000FC2137F65C207C35050AB683679717C919
:100A4000F5D93F319A6361787E779BDCBCFF788B68
:100A5000B1095ACE9BF3F9D1CD7908FF6713EFB0F6
:100A60007BA2C3CBE9D1CD251E5C7CF874F173F277
:100A7000EEF3D52F28C929FD3B9A5C5FDC0154DADF
:100A800095629B86513C05C09BAFD7CC2DC46CF3BF
:100A9000F9EAE2EAFD3FAE92AFEF3F5E7EFA8A3EB0
:100AA0001FE2C7DBABCFF0916F215A9916C8EB0A52
:100AB000785D212F387D7FF621393FBBBB4432CC96
:100AC000EAF6CBD997DBE4F6EEFAF61738B9BDC2F1
:100AD00093F8158B8D1EEA1FAAD0A9F9D58D092E82
:100AE000E90D5380019BC6FDCDD97472FAAFE9D1EF
:100AF000EADF70CD735CAF787D816BB00FDA5CE2BA
:100B000006DA30DA5CE106DA4BDABCC3CD42E3FF49
:100B1000441B4DE06FB8893481BFE366A9717E261E
:100B2000361AE7036D10E775101AA03CA5BE7D3696
:100B30009FCFE1C647935445D3C532A7BCDF1522EA
:100B40008226FF1E1EACB1F4F3487FF83CCC3E1267
:100B50004DB085323391B9567A40C6B1E1ACC92E59
:100B60007556A08DBF04A604CBB98EBA48ABA0AA17
:100B7000BB008C3DC08011408CE3C01690CD064F69
:100B80003B096BB63D1534E03DC089070A06B757EF
:100B900082B2583B0B36751B8019FCD5ECA5C2D32D
:100BA0009CBED327C5190350FFD4613E80FE620B63
:100BB0001782A23DED103AD5D7E46E8A9D5D032BD6
:100BC00004459367EFE3AF943A8834DC5454816969
:100BD000382C3E18DD050F4882266DC1E402D1B6DF
:100BE000754BD9C21CB4023298EA680AF22E85F716
:100BF000E64157071429B0EF2507E70EE47D05BE4F
:100C000026F3C0CC11DC5883D31CF719064A4F6673
:100C100068ACE0BE01185E252D05E448EED8CC6135
:100C2000593F0A739B007B5FAEAACDB1ED946D6F07
:100C3000CC25FFDEB9AE062D7FECC80C1008306065
:100C4000B3C30ED57CC596D6C48D7039F8AEAB98BB
:100C50006C271B8D388F8600A082BE716F521C4698
:100C60000DC4A08EF1A96014499FD14E5746A05CD7
:100C70000F5F0BA5D2AD08A0B3815C64140624AF4E
:100C8000A5426B525007E67D819D152063EA0E74E4
:100C90005424C3178F02358133A56F23ECD2362736
:100CA00063D7D0D8065CA3F8A9980960D56E8AFAF4
:100CB00089FBFE8F60E569C0CF41F7A2A8B2181D7D
:100CC00080DDF301361EFE81AC1A2E1A383FD35157
:100CD0008537759F17143DADF5376DBD056196706D
:100CE000F514DFB681AC0BB704610B745C6CFD3E90
:100CF0000BFD283456F42C6083A20635A0256373BF
:100D0000706B01F6A4133CC9A280649401BDC1A814
:100D1000836B33876925F41D0C9CC1DD8217B20EED
:100D2000E9020821CBBE34DF8C738065DD9A710641
:100D30007555408CFC9662901DFD2141EDC85D5DAE
:100D4000079B945EC72FC331D917DFA40EC4BBF530
:100D50000804A50AB468C6C355D7171219128754D8
:100D6000AD04F5EF7795EA1B4CD782FD9E822D16D8
:100D7000885FD32EDBE5F59605FD035744346A857D
:100D80008EA4AF1E8030060DEEEEBDEFCA1D80F1C1
:100D9000B21B415451100CD1C9A11080DE52B109CF
:100DA000CCDD408C635A5D1510061F81407A5F9838
:100DB000E86625B4A6A632D0F509B70DA32EF63401
:100DC000F804F11572E43D96141B1C64A81FB87159
:100DD000A5E9B00DB57A669C73D3A7B017AD20888E
:100DE000B05565708C470B5B4251F421D115698B6E
:100DF000E2C612FE4071822A6507C029948EC8ECB3
:100E00005E582143F6DA9BD460FA820A623E5B4563
:100E1000116543BD89291DF2268EC83E6013C74B5C
:100E200058CF5F5FA98368207C081E82EB86D5AF10
:100E30002F1506D52A13A3B6788D8A3CD4DFBA5E67
:100E4000473763A680E346C1A776DF937B12D64679
:100E50006E6AFC2DA437E9C68E008B1FDB270F06B8
:100E6000234CF1506BB5F286F2038CD46B82033ABB
:100E7000E1D71CA3E17307E52AD5951D59417ED51D
:100E800033157A20CD5EF09BB12A6A1020F0F9F775
:100E90005ED114937AEBEFDD5A63E845E2B81F8721
:100EA000B11B7829703F3BBF5A79E3A201E55D0D84
:100EB000EDEC769F873F8D02F4D8CD5F12A37E576D
:100EC00039F35E2B79E6462C1EA89DB5B0399C20DF
:100ED00028989C2790605C5EB14C96E0E5A6FDFFEB
:100EE0000336768C89EEE0B8E0FF32B27EDFC88E42
:100EF000E7FEB048CBDB5CAECF321AD167A81478DE
:100F00000148C11F4CAEB0C973A1D90C700E0B6063
:100F1000D0DEFE2111843E86D782F908A0A9E850D0
:100F2000DFBCA75E7F0AE2EB7931EC537FC72C561A
:100F3000D48E4240A38276197335AD9C2DABBED4BE
:100F40003FEA571E8CAC5DE7396A4B79E40655F9E8
:100F50002A1AC5B5A11A0E3A7BCF9989A7A453D7EF
:100F6000ABEEDF1FBB54F6F495DF7F3AE7C952DBE7
:100F70000C1F1CD3FA81817A4A2A9DF98F16BD7FF6
:100F800088DD85FEF32474688FD393D9F4647A1CCA
:100F900045CBE3ED6629C2F57DB89CBCFE1756BD76
:100FA000A41B640A000020002300260029002C0056
:100FB0002F003200000100000301060109010F4764
:100FC00000440045008001354800440045002001F0
:100FD0000D88008000810080000E8A008000810062
:100FE00020000F8C008000810008000CB300B000CE
:100FF000B10080033EB400B000B10020032398008C
:10100000900091008000249A00900091002000251B
:101010009C009000910008003BA800A000A1008067
:10102000003CAA00A000A10020003DAC00A000A14F
:101030000008005B28012001210180005C2A0120BA
:1010400001210120005D2C01200121010800040084
:101050000000040404040704000002040002040267
:101060000400070402070400000204040204000054
:10107000040407040002040404000404000404013E
:101080000704000402000000000000000600020245
:101090006617044E10650A02521064400271106314
:1010A000400354106240036310611F0757106040F3
:1010B0000363105F0B025E105E400360105D40032F
:1010C00063105C1C0766105B400271105A14046DBB
:1010D0001059400271105810037310571104761004
:1010E0005611047A10550D027E10540B01851053D1
:1010F000400180105212048110510B0185105010D4
:101100000286104F150388100040028B104E0E020D
:101110008D104D09018F104C0600000028292A2B44
:101120002C2D2E2F505152535455565711241FBE5B
:10113000CFEFD1E2DEBFCDBF00E00CBF14BE0FB6D3
:10114000F894A89580916000886180936000109267
:1011500060000FBE12E0A0E0B2E0E4E8F5E700E0D6
:101160000BBF02C007900D92AA32B107D9F723E056
:10117000AAE2B2E001C01D92A739B207E1F70E94CE
:101180006D260C94C03A0C940000CF93DF93CDB73A
:10119000DEB76E970FB6F894DEBF0FBECDBF0E94CC
:1011A0005A266B017C019E012F5F3F4F1901AE0152
:1011B000475F5F4F5B8B4A8B80912602882309F43F
:1011C00034C50E945A26C61AD70AE80AF90AF894C2
:1011D00080912602882351F08FEF80932602789425
:1011E0000000F894809126028111F9CF78940E9432
:1011F0005A26A7019601260F371F481F591F288F0F
:10120000398F4A8F5B8F81E08093260280914C0258
:10121000882309F440C010924C028FEF89839BED24
:10122000E92E90E1F92E69E373E2C1010E945D119C
:101230008C01892B81F1D80156968C9182FFF3CFD6
:101240000E945A26F894F80137892689422F4B7F4D
:10125000468B78949F938F937F936F931F923F93C6
:1012600021701F922F9389811F928F93FF92EF928B
:101270000E94C0312DB73EB7245F3F4F0FB6F894A0
:101280003EBF0FBE2DBF69E373E2C1010E945D1135
:101290008C01892B81F680914D02882309F11092EF
:1012A0004D028FEF898306ED10E16BE774E3C10116
:1012B0000E945D11FC01892B99F0958D868D981304
:1012C000F4CFF894858D968D891709F48FC578949D
:1012D0006BE774E3C1010E945D11FC01892B69F782
:1012E00080914702882309F456C0109247028FEF7D
:1012F000898B8CE0B82E63E179E1CE0141960E94A2
:101300005D114C01892B09F446C0D40157968C918C
:10131000579780FFF0CFF894F401448055806680A1
:10132000778087898E7F878B789456968C918130D1
:1013300009F4E5C308F4BDC3823009F47EC38330E9
:10134000D1F6A9881F86188A9E01215F3F4F42E08F
:1013500061E0F401848995890E9469198F859889D3
:10136000382F292F3D8B2C8B790100E010E0B40140
:10137000605F7F4FC12CA3019201C4010C960E94B3
:1013800053173C8932FFB7CF809127028111B3CF29
:101390008CE10E94EB3780914602882389F11092FC
:1013A00046028FEF8B87A2E0DA2EBDE2EB2E18E02B
:1013B000F12E6AE574E1CE010B960E945D118C015D
:1013C000892BF1F0D80152968C9182FFF2CF80FFE9
:1013D00012C0C8010E943435F801D28AE982FA822B
:1013E000910142E060E0848595850E946919C801F9
:1013F0000E947915DECF6B85C8010E94BE15D9CF3A
:1014000080914502882309F45AC0109245028FEF5B
:101410008B8777247A94FDE14F2E62EA71E1CE0149
:101420000B960E945D118C01892B09F448C0D801EC
:1014300050968C9182FFF1CFF894F80184809580CA
:10144000A680B780F488108A148A78948085918564
:10145000A285B385881A990AAA0ABB0AD801FF2077
:1014600089F052968C91F801E80FF11D758A168A61
:10147000178A8D5FF801828B8E32D8F4FA94D801E6
:10148000F110EFCF51968C91882309F477C2813007
:1014900009F462C3823009F457C4D80152968C9182
:1014A00090E08E970CF4B9CF6B85C8010E94CD38BF
:1014B000B4CF6B85C8010E94CD38FA94E0CF8091FB
:1014C0005102882309F45FC0109251028FEF8B877D
:1014D00012E0A12E03E2E02E8AE6F82E94E0B92E67
:1014E00020E4C22E38E0D32E6DE97EE2CE010B96C9
:1014F0000E945D118C01892B09F445C0F801828995
:1015000082FFF2CF80FF3AC0C8010E943435D80173
:101510005296AC925297E9821A821C96ED91FC91F8
:101520001D97A10162E080810E946518F982BA824C
:10153000D8011C96ED91FC911D97A10162E080817C
:101540000E946518F982CA82D8011C96ED91FC911F
:101550001D97A10162E080810E946518E982DA820C
:10156000D8011C96ED91FC911D97A10162E080814C
:101570000E946518C8010E943730B6CF6B85C8013C
:101580000E945630B1CF809148028823E9F0109232
:1015900048028FEF89830FE910E164E87BE1C10124
:1015A0000E945D11009781F0FC01208D2F3FA9F76B
:1015B000F8942685211104C3789464E87BE1C10185
:1015C0000E945D11009781F7809149028823D9F12B
:1015D000109249028FEF89830AE910E164EC7EE101
:1015E000C1010E945D11009771F1DC011E962C91E2
:1015F0001E9723FFF3CFF894FC012685277F2687CB
:1016000078949C01265E3F4F3F932F9350968C9188
:101610008695869586951F928F9389811F928F93C9
:101620001F930F930E94C031EDB7FEB738960FB6E7
:10163000F894FEBF0FBEEDBF64EC7EE1C1010E94D5
:101640005D11009791F680914E02882309F446C0FF
:1016500010924E028FEF898300E910E16AEE74E286
:10166000C1010E945D11FC01892BC1F1848D80FFB5
:10167000F5CFF89494812581368147815489658915
:101680007689A789B08DF18CE28CD38C848D8E7F86
:10169000848F7894DF92EF92FF92BF93AF937F9302
:1016A0006F935F934F933F932F939F9389811F92E3
:1016B0008F931F930F930E94C0312DB73EB7205FC9
:1016C0003F4F0FB6F8943EBF0FBE2DBF6AEE74E2D7
:1016D000C1010E945D11FC01892B41F6A895809102
:1016E0007302882329F080E48093600010927302D3
:1016F00010913403112309F46DC000912A0200FDFA
:1017000012C0153008F466C0B0907402CB2C8BEF79
:101710008B0D8C3308F4B0C2EEE7CE1609F41AC470
:10172000016000932A02412F50E06EE770E084E7E9
:1017300092E00E94913A009739F00E7F00932A02BE
:101740008457924011E0180F01FD0CC0902F926059
:1017500090932A0289E395E09F938F930E94C03172
:101760000F900F90B12EDD24DA9480E0EB2CF12C59
:1017700018C090E0402F50E0481B590BB701680F8C
:10178000791F6C587D4F8C589D4F0E94A73A10923C
:101790002602802F9FB7F89420913403121761F02E
:1017A0009FBF10913403012F0B1919F79FB7F894BD
:1017B000209134031213F4CF009334039FBFF1E060
:1017C000DF1208C089E395E09F938F930E94C03198
:1017D0000F900F900E945A266B017C01288D398D45
:1017E0004A8D5B8D621B730B840B950B80903302CB
:1017F00090903402A0903502B09036023FEF831AE9
:10180000930AA30AB30A8092330290923402A09200
:101810003502B092360240902F0250903002609014
:10182000310270903202460E571E681E791E409299
:101830002F02509230026092310270923202611592
:10184000710541E08407910508F0F4C19B01AC01EA
:101850000E94103ADC01CB0181509F4FAF4FBF4F28
:10186000892F9A2FAB2FBB2740912B0250912C022E
:1018700060912D0270912E02840F951FA61FB71F35
:1018800084179507A607B70718F48FEF9FEFDC01C1
:1018900080932B0290932C02A0932D02B0932E02E2
:1018A00040916F02509170026091710270917202CA
:1018B0005C546B437B4F2F2DC416D506E606270BD1
:1018C00027FD7ACCBF93AF939F938F937F926F92B4
:1018D0005F924F92BF92AF929F928F9283E091E17D
:1018E0009F938F930E94C0316DB77EB7625F7F4F29
:1018F0000FB6F8947EBF0FBE6DBF80916F029091BE
:101900007002A0917102B0917202C816D906EA065F
:10191000FB0698F480916B0290916C02A0916D028D
:10192000B0916E020196A11DB11D80936B02909340
:101930006C02A0936D02B0936E02C0926F02D092BF
:101940007002E0927102F092720210922B021092D9
:101950002C0210922D0210922E0210922F02109241
:101960003002109231021092320210923302109221
:10197000340210923502109236021ECC82E3898323
:101980001A820E945A266B017C01910142E061E0BB
:10199000F801848595850E9469190E945A26DC0108
:1019A000CB018C199D09AE09BF0981329340A10575
:1019B000B10508F0F7C0998197FD2EC1C818D90864
:1019C000EA08FB08D80153968C918823C1F02FEFC9
:1019D000280F41E050E002C0440F551F2A95E2F75E
:1019E000052E000C660B770BC40ED51EE61EF71EE7
:1019F00004C0F694E794D794C7948A95D2F7BFEFC2
:101A0000CB16D104E104F10408F064C12A8130E06E
:101A1000220F331F892F90E0982F8827990F822B50
:101A2000932BF8012289E20FF11DC58A868B978BD3
:101A30002D5FD80152962C9330CDA98881E08983FF
:101A40001A821B821C82910143E061E0848995899E
:101A50000E94691969817A818B819C810E94203A58
:101A6000272F382F492F55272C8B3D8B4E8B5F8B83
:101A700037E039831A82910142E061E0D401549643
:101A80008D919C9155970E946919EC88FD880E896B
:101A90001F8900271127B401605F7F4FCA80A3010F
:101AA0009201C4010C960E945317BC89B0FF23CC4D
:101AB0006BCCA9881B861C861D861E869E01255F11
:101AC0003F4F44E061E0F401848995890E946919DF
:101AD0006B857C858D859E850E94203AD62EF72EBB
:101AE000B401605F7F4FC12CED2C8C01A3019201EA
:101AF000C4010C960E945317D2FEFDCB45CCA98899
:101B0000B9821A821B821C82910144E061E08489BF
:101B100095890E94691969817A818B819C810E94D3
:101B2000203A6B017C01BFE0B9831A82910142E047
:101B300061E0F401848995890E9469198701760121
:101B40001127B401605F7F4FCA80A3019201C401D5
:101B50000C960E945317CFCB8FE789838EEF8A8331
:101B60000E945A266C8B7D8B8E8B9F8B910142E05D
:101B700060E0F801848595850E9469190E945A26C3
:101B80006B017C01DC01CB012C893D894E895F8989
:101B9000821B930BA40BB50B81329340A105B105B9
:101BA00008F4A5C0D80152968C91F801E80FF11DF8
:101BB000758A92E0968B178A8D5FF801828B6DCCC7
:101BC000FC01318D308F7894AC01415F5F4F5F93A2
:101BD0004F931F922F9387891F928F9389811F9212
:101BE0008F931F930F930E94C031EDB7FEB73A96C3
:101BF0000FB6F894FEBF0FBEEDBFCFCC2A893B894C
:101C0000E217F30709F0E3C0809590E02A8530E001
:101C10008217930709F40AC1D80152968C91F801F2
:101C2000E80FF11D758A93E0C5CFC88ED98EEA8E74
:101C3000FB8EE9CA6115710550E18507910508F031
:101C400024CE8B019C0101501F4F2F4F3F4F552732
:101C5000432F322F212F0E94103ADC01CB014091FB
:101C60002B0250912C0260912D0270912E02840F54
:101C7000951FA61FB71F04CED09075028D2D807FB3
:101C8000803109F049CD1B1508F4A4CD8B2D90E0CF
:101C9000FC01ED58FD4F20812E3709F03DCDAC0100
:101CA0004F585D4F4A01FC01EE58FD4F9081DA011B
:101CB0008C91292F30E07901F82A6DEF6B0D84E7C4
:101CC00092E00E947026E816F90609F445C1C0901A
:101CD000740222CDF8018289E80FF11D758A91E026
:101CE000968B178A8D5FD80152968C93D6CB80EC59
:101CF00089831A82910142E061E0D8011C968D919E
:101D00009C911D970E94691949812A81942F9227DD
:101D1000892F82958F709827892F86958695892798
:101D2000982F9695892780FD95C046FFA3C0F8019E
:101D30008289E80FF11D758A25E0268B178A8D5F51
:101D4000D80152968C93A9CBD8011C96ED91FC91A9
:101D50001D976480B281BC8B538040E06B2F752D42
:101D6000862D0E94E9180E945A266B017C01E0E151
:101D7000CE0ED11CE11CF11C0E945A262F2DC61636
:101D8000D706E806290B27FFF7CFF89441E06C89C6
:101D9000752D862D0E94E9180E945A266B017C0140
:101DA0007894D101EAE01D92EA95E9F7F4E8F98325
:101DB00023E22A8391014AE061E0D8011C968D91CB
:101DC0009C911D970E946919FE01339685E09191BF
:101DD000892728E030E005C0880F2150310909F437
:101DE0000DCF87FFF9CF880F8425F7CF54896589F8
:101DF00090892189328943898F5F858F78946F9389
:101E00005F934F933F932F939F9389811F928F935B
:101E10001F930F930E94C0314DB75EB7465F5F4F6F
:101E20000FB6F8945EBF0FBE4DBF3FCA898584FFD1
:101E300018C08B8187FD60C0D80152968C91F80143
:101E4000E80FF11D758AB4E0B68B178A8D5FF80133
:101E5000828B23CBF8018289E80FF11D758A93E00C
:101E60003FCFD80152968C91F801E80FF11D758A89
:101E7000B5E0EACFC818D908EA08FB08F8013389A9
:101E80003323C9F08FEF830F61E070E002C0660F6B
:101E9000771F8A95E2F7CB01092E000CAA0BBB0B2A
:101EA000C80ED91EEA1EFB1E04C0F694E794D79410
:101EB000C7943A95D2F77FEFC716D104E104F10435
:101EC00008F03FC0842F90E0AC01542F4427550FF9
:101ED000550FF4E02F9FC0011124842B952BD801BE
:101EE00052962C91F801E20FF11DC58A868B978BD3
:101EF0002D5FF801228BD1CAC818D908EA08FB085F
:101F0000F1E5CF16F5E5DF06E104F104D0F42C810C
:101F100030E0220F331F90E0982F8827990F822BF3
:101F2000932BD80152963C91F801E30FF11D2F81BC
:101F300026952F73258B868B978B3D5FF801328B0F
:101F4000ACCAD80152968C91F801E80FF11D758A40
:101F500091E030CE11E006CC802F8D7F80932A0255
:101F600080910802D81202C181E08D0D8F708061CE
:101F700080930802B6E78B16B2E09B0609F008F4DE
:101F8000BEC0E6E7F2E0BE8ECDB6DEB68F010F5FD3
:101F90001F4F2081222309F4E6C0E8E3F5E0849195
:101FA000281708F0E0C030E0220F331F220F331F44
:101FB000220F331FF901E752FD4FE4914DB75EB791
:101FC00064E0E69F4019510911240FB6F8945EBFF2
:101FD0000FBE4DBF8DB79EB70196F901E552FD4F7B
:101FE0004491F901E452FD4F65917491FB01640F36
:101FF000711DAC01DD8ACC8A9D8F8C8F6E177F0797
:1020000009F482C08016910608F46EC0A491A53030
:1020100028F1A73009F068C02801BFEF4B1A5B0A0E
:10202000D801AC9082010A0D111D8016910608F4AA
:102030005BC0B12CC12CD12CDA01AD92BD92CD92F6
:10204000DC921397612C712C14964D925D926D92D7
:102050007C921797485F5F4F3196D0CF7A0184E02A
:10206000E80EF11C68019FEFC91AD90AD8011C912A
:10207000912F9F77492E512C612C712C012F0076C6
:102080000036A9F117FF3EC086010F5F1F4FD80130
:1020900011978C91440C551C661C771C440C551CE4
:1020A000661C771C440C551C661C771C440C551C84
:1020B000661C771C440C551C661C771C440C551C74
:1020C000661C771C440C551C661C771C982F9F7748
:1020D000492A87FDDACFDA014D925D926D927C92AA
:1020E0001397A70131968ACF87E00E94EB37B0EEB5
:1020F0004B2A55245A94652C762CC4CFBE8CDD24F3
:10210000D39433CB8601E7CFCC88DD888C8D9D8D31
:1021100040912702442331F0F901E652FD4FE4914A
:10212000E0FF11C022523D4FF90125913491F90190
:1021300019950FB6F894DEBE0FBECDBE0815190571
:10214000E8F6F80121CF809128021F928F93E2E1F7
:10215000F1E1FF93EF930E94C0310FB6F894DEBE19
:102160000FBECDBEEBCF85E00E94EB371B2DF2CA30
:102170000F931F93CF93DF938C0180913F02909137
:102180004002892B09F04BC060913E0270E0623042
:1021900071052CF482E080933E0262E070E0E091F1
:1021A0003A02F0913B024DB75EB741505F4F442772
:1021B0005A959F01C0E0D0E0C901860F971F4817CC
:1021C000590730F121969C01C115A4E0DA07A1F767
:1021D0008E1B9F0B0E949D31D0934002C0933F0203
:1021E00090933D0280933C020E94D828F8018081A0
:1021F0009181A281B3818093410290934202A09386
:102200004302B0934402DF91CF911F910F91089543
:10221000209711F0C901DCCF80E10E94EB378DE0FF
:102220000E94EB37CF932091380230913902232B53
:1022300091F4FC01C0818C2F90E0880F991F880FCA
:10224000991F0E949D319093390280933802C09368
:102250003702CF9108958AE00E94EB3780913F02C8
:10226000909140029F938F9321E03091270231118A
:1022700001C020E01F922F93209144022F932091C0
:1022800043022F93209142022F93209141022F93DA
:1022900021E0892B09F420E01F922F9384EF90E135
:1022A0009F938F930E94C0318DB79EB70C960FB647
:1022B000F8949EBF0FBE8DBF0895CF93DF93EC01BE
:1022C000988140913702A0913802B09139020BC039
:1022D000FD0184E0989FE00DF11D112420813181E2
:1022E0002617370741F09F5F941790F380E090E046
:1022F000DF91CF910895988382819381DF91CF916F
:102300000895FC01808982FD19C08460808B109241
:10231000260281E080934502448155816681778160
:1023200080859185A285B385840F951FA61FB71F51
:1023300084839583A683B78381E0089584898F5F22
:10234000848BE5CFFF920F931F93CF93DF93EC0124
:10235000F88483E08F1508F145E450E062EA71E10A
:1023600088810E9491288C0181E891E1F801938392
:10237000828365EA73E38C810E94C028F801958707
:102380008487FC01858180FF0BC0F801F18ADF9111
:10239000CF911F910F91FF90089583E20E94EB3738
:1023A00082E20E94EB378F929F92AF92BF92EF92A0
:1023B000FF920F931F93CF93DF931F921F92CDB77E
:1023C000DEB77C016AE574E1FC0180810E94C028CF
:1023D0008C0189EB89831A820E945A264B015C0189
:1023E0009E012F5F3F4F42E061E0F80184859585B3
:1023F0000E9469190E945A26F80121892F93208989
:102400002F932A811F922F9323891F922F93278521
:102410002F9326852F93DC01CB0188199909AA09EE
:10242000BB09BF93AF939F938F93BF92AF929F923D
:102430008F92F70180811F928F9382EC90E19F939E
:102440008F930E94C0310FB6F894DEBF0FBECDBF90
:102450000F900F90DF91CF911F910F91FF90EF9010
:10246000BF90AF909F908F9008954F925F926F9220
:102470007F928F929F92AF92BF92DF92EF92FF92E4
:102480000F931F93CF93DF931F921F92CDB7DEB7A9
:102490007C01FC01D0806AE574E18D2D0E94C0288A
:1024A0008C01F70180859185A285B385892B8A2BC4
:1024B0008B2B99F1C8010E943435F70184819581F5
:1024C000A681B781F80184839583A683B783F7013A
:1024D00080859185A285B385F80180879187A28741
:1024E000B38781E0828B118A108A17861686138A39
:1024F000C8010E9486350F900F90DF91CF911F91F8
:102500000F91FF90EF90DF90BF90AF909F908F90D2
:102510007F906F905F904F900895C8010E9434356E
:10252000F801128A8DE289831A820E945A264B0191
:102530005C019E012F5F3F4F42E060E0F80184851F
:1025400095850E9469190E945A262B013C0181E25F
:10255000F82E99EBE92E03C0FA94FF20C1F0E9822E
:102560001A829E012F5F3F4F42E061E0F8018485AF
:1025700095850E9469198A818F7749F0813260F7C9
:102580006D2DC8010E94BE15FA94F110E8CFF80134
:102590008389882331F06D2DC8010E949815F801B8
:1025A0008389F80191899F9390899F939A811F92C3
:1025B0009F931F928F9387858F9386858F93D301E7
:1025C000C20188199909AA09BB09BF93AF939F93C8
:1025D0008F93BF92AF929F928F921F92DF9282EC65
:1025E00090E19F938F930E94C0310FB6F894DEBFA5
:1025F0000FBECDBF80CF8F929F92AF92BF92FF92BE
:102600000F931F93CF93DF938C016CE873E1FC0170
:1026100080810E94C028EC010E9434358F8D98A1E2
:10262000892B09F058C0F80104811BA1FF24F39401
:10263000002339F16C897D898E894F2D0E94E9181C
:1026400021E001111CC014FB882780F991E0892743
:10265000281741F08F89988DA98DBA8D892B8A2BE7
:102660008B2B89F410711F291BA3DF91CF911F9130
:102670000F91FF90BF90AF909F908F90089520E0B2
:10268000E2CFF12CD7CF0E945A268F88988CA98C44
:10269000BA8CDC01CB01880D991DAA1DBB1D888B4E
:1026A000998BAA8BBB8B8C839D83AE83BF8383EF77
:1026B00096E29B838A83107114601F291BA3CE01AD
:1026C000DF91CF911F910F91FF90BF90AF909F909E
:1026D0008F900C94863582E10E94EB37CF93DF9385
:1026E000EC016CE873E188810E94C028F894FC0139
:1026F000278D30A1232B69F44C815D816E817F8110
:10270000FC01438F548F658F768F7894DF91CF9142
:10271000089584E10E94EB37CF92DF92EF92CF933E
:10272000DF93EC0161E088859985AA85BB85892BBB
:102730008A2B8B2B09F460E08C810E9408256B01A9
:10274000E82E44E250E06CE873E188810E94912811
:10275000FC01C48AD58AE68A21E0488559856A85C4
:102760007B85452B462B472B09F420E04C855D8566
:102770006E857F85452B462B472BB1F430E0232B0C
:10278000FC0123A3488959896A897B89478B508F2B
:10279000618F728F6AE070E04F96DF91CF91EF907A
:1027A000DF90CF900C94222930E1E9CFCF92DF92D5
:1027B000EF92FF920F931F93CF93DF938C016CE8FE
:1027C00073E1DC018C910E94C028EC010E943C293D
:1027D000FC01D8011496CD90DD90ED90FC901797F8
:1027E000C282D382E482F58218964D915D916D91FB
:1027F0007C911B974683578360877187F894118279
:1028000010828F8D98A1892B81F0A9A1BAA1ED9397
:10281000FC93FAA3E9A37894DF91CF911F910F91D4
:10282000FF90EF90DF90CF900895FAA3E9A3F8A36B
:10283000EF8F8BA182FD25C0C88AD98AEA8AFB8ADC
:10284000982F94609BA381FD10C0CE010E94343567
:10285000CC82DD82EE82FF8283EF96E29B838A83C5
:10286000CE010E9486357894D7CF4C815D816E81F0
:102870007F81872F4C155D056E058F0987FFE5CF9A
:10288000F2CF488959896A897B89972F4C155D0554
:102890006E059F0997FFD0CF83E10E94EB37FC01C3
:1028A00092899460928B1092260281E08093460276
:1028B00080E008950F931F93CF93DF938C0146E43C
:1028C00050E06AE574E1FC0180810E949128EC01EE
:1028D0008FE494E19B838A8365EA73E3F801848142
:1028E0000E94C0289D878C87DF91CF911F910F9107
:1028F0000895FC014481558166817781208580811E
:102900000C945029EF92FF920F931F93CF93DF9374
:102910007C016CEF74E1DC018C910E94C0288C0179
:102920000E943C29EC01F70184819581A681B78141
:102930008A839B83AC83BD83808591859F838E83AF
:10294000F89419821882D80151968D919C915297D2
:10295000892BB9F15396ED91FC915497D183C083A3
:102960005496DC93CE93539780E090E07894892B33
:1029700039F4DF91CF911F910F91FF90EF9008955F
:10298000C8010E943435D80112968D919C911397FD
:10299000875F9042F1F08A819B81AC81BD8122E703
:1029A00030E2F8013383228384839583A683B7833F
:1029B000C801DF91CF911F910F91FF90EF900C9480
:1029C0008635F801D48BC38BD28BC18B81E090E02C
:1029D000CDCF8A819B81AC81BD81F8014481558135
:1029E00066817781272F481759076A072B0B27FF26
:1029F000D6CF80E20E94EB37CF92DF92EF92CF9357
:102A0000DF93EC01488559856A857B852C858C810F
:102A10000E9450296B01E82E45E150E06CEF74E113
:102A200088810E949128FC01C086D186E28688892F
:102A30009989908B87878C899D89AE89BF89838787
:102A40009487A587B68782E790E29383828368E0C4
:102A500070E0CF014196DF91CF91EF90DF90CF9062
:102A60000C942229DF92EF92FF920F931F93CF9342
:102A7000DF93EC01D88883E08D15B0F165EA73E34C
:102A800088810E94C0287C018AE090E00E949D31EC
:102A90008C0161E08C810E94B018F8016083718321
:102AA000828360E088850E940825F801638374832F
:102AB000858360E08C850E940825F8016683778312
:102AC0008087D186F7018581982F967081F4F70170
:102AD0001183008382608583DF91CF911F910F91D5
:102AE000FF90EF90DF9008958BE10E94EB370E94FA
:102AF00066190F931F93CF93DF93EC01F8940E9414
:102B00005A26088519852A853B85DC01CB01800F73
:102B1000911FA21FB31F8C839D83AE83BF83CE0101
:102B20000E9486357894DF91CF911F910F9108957F
:102B3000CF93DF93EC0144969F938F938B891F92E1
:102B40008F938F858F938E858F931F926F938DEBCD
:102B500090E19F938F930E94C0311B8A8E859F8541
:102B600001969F878E878DB79EB70A960FB6F89409
:102B70009EBF0FBE8DBFDF91CF910895DF92EF9280
:102B8000FF920F931F93CF93DF93CDB7DEB72997B3
:102B90000FB6F894DEBF0FBECDBF8C01F62E9E019E
:102BA0002F5F3F4F89E0F90111928A95E9F782EF93
:102BB000898349E061E0F801848595850E9469195F
:102BC000F801838990E09C012C5E3F4FE20FF31FD8
:102BD0003B81232F207F21F1203F11F12FEF248310
:102BE000238322832183F801E80FF91F248BF80146
:102BF00083898B5F838B8E3208F05EC0F8018289F7
:102C000081FD4FC029960FB6F894DEBF0FBECDBF31
:102C1000DF91CF911F910F91FF90EF90DF9008957A
:102C20004D81242F207FC9F52F81522F507F11F025
:102C3000503FA1F65885503989F659855F77E52EC2
:102C400050E25E1558F2D801A80FB91F5A81549668
:102C50005C938C8181838E818283822F90E03F718F
:102C6000BC01660F771F62957295707F7627607F33
:102C70007627362B3383880F991F880F991F80760C
:102C80004F71482B4483F80183898B5F838B4EEF10
:102C9000D42EDE0C8E32B8F012C0203F09F09ECF49
:102CA000C3CFC8010E943435F80182898B7F828BA3
:102CB000C8010E947915A6CF8EEFD82EE12C6F2D7A
:102CC000C8010E949815FEE1FE1530F4F8018089D4
:102CD00091890196918B808BFEE1FD1508F48ECFD2
:102CE0001092260281E0809346028CCFAF92BF9271
:102CF000CF92DF92EF92FF920F931F93CF93DF93C8
:102D0000CDB7DEB77C01ADB6BEB6FC01C0806AEDC2
:102D100076E18C2D0E94C028F701648140855185A1
:102D2000D4842DB73EB72D1931090FB6F8943EBFA4
:102D30000FBE2DBFEDB7FEB731967F018F012D2D50
:102D4000FC0180810E94DB17FF92EF921F92DF92BD
:102D50001F92CF9287EC90E19F938F930E94C03196
:102D60002DB73EB7285F3F4F0FB6F8943EBF0FBE5A
:102D70002DBF0FB6F894BEBE0FBEADBEDF91CF9192
:102D80001F910F91FF90EF90DF90CF90BF90AF9089
:102D90000895CF93DF93EC016AED76E188810E947C
:102DA000C028488559856C81FC018081DF91CF91D5
:102DB0000C946518EF92FF921F93CF93DF93EC0171
:102DC0008C85182F1F7741E050E06AED76E188810D
:102DD0000E9491287C018C819D81AE81BF81892BCD
:102DE0008A2B8B2BF1F48091BC0082FD10C061E036
:102DF00089E10E94082561E088E10E94082510927F
:102E0000B90088E48093B80084E08093BC00812FEF
:102E1000880FF7018083DF91CF911F91FF90EF9092
:102E2000089581E30E94EB370F931F93CF93DF93B5
:102E30008C0163E179E1FC0180810E94C028EC01F2
:102E40000E943435F80184819581A681B7818C83F5
:102E50009D83AE83BF8380859185A285B385888756
:102E60009987AA87BB87892B8A2B8B2B29F4DF9123
:102E7000CF911F910F91089584859585A685B7857B
:102E80008C879D87AE87BF8780899189A289B38906
:102E9000888B998BAA8BBB8BCE01DF91CF911F9131
:102EA0000F910C9486354F925F926F927F928F9222
:102EB0009F92AF92CF92EF92FF920F931F93CF9377
:102EC000DF93EC014B01270138011F92CF927F92D3
:102ED0006F925F92EF925F934F933F932F931F9266
:102EE000AF928CEC90E19F938F930E94C0318DB78D
:102EF0009EB70E960FB6F8949EBF0FBE8DBF888109
:102F00009981AA81BB81E816F9060A071B0750F0D0
:102F1000F40180819181A281B3818E159F05A00764
:102F2000B10720F480912702882379F0DF91CF91B7
:102F30001F910F91FF90EF90CF90AF909F908F9047
:102F40007F906F905F904F9008958DE10E94EB37D6
:102F5000CF92DF92EF92FF926B017C0109C00E9439
:102F60005A26292F6C157D058E052F0927FF09C0CC
:102F70008091BC0087FFF3CFFF90EF90DF90CF9060
:102F8000089580E30E94EB3724EA2093BC000E945E
:102F9000A8178091B90090E0A0E0B0E080319105E1
:102FA000A105B10521F00897A105B10509F408951F
:102FB0008FE20E94EB377F928F929F92AF92BF92E7
:102FC000CF92DF92EF92FF920F931F93CF93DF93F5
:102FD000782EC62F942EB52E822E0E945A266B0173
:102FE0007C0120E8C20E28E3D21E21E0E21EF11C83
:102FF000C701B6010E94C4177092BB0084E8809399
:10300000BC00C701B6010E94A817AA24AA94AC0E5E
:10301000CC23B1F0C92DDB2DB12C8FEFA81AB80A43
:10302000AC0EBD1E94E8992E89918093BB009092BE
:10303000BC00C701B6010E94A817AC16BD06A1F7D7
:10304000C701B6010E94C417872D81608093BB0021
:1030500084E88093BC00C701B6010E94A817DFEF87
:10306000D80D882009F15801CD2F84EC982ECC235F
:1030700069F09092BC00C701B6010E94A817809128
:10308000BB00F50181935F01C15099F7F801ED0F85
:10309000F11DEF0184E88093BC00C701B6010E94D6
:1030A000A8178091BB00888384E98093BC00DF91DE
:1030B000CF911F910F91FF90EF90DF90CF90BF9035
:1030C000AF909F908F907F900895BF92CF92DF92A4
:1030D000EF92FF920F931F93CF93DF93D82FC62FBA
:1030E000B42E152F0E945A266B017C0120E8C20ED7
:1030F00028E3D21E21E0E21EF11CC701B6010E94A6
:10310000C417D093BB0084E88093BC00C701B6010C
:103110000E94A8170FEF0C0FCC23A9F0CB2DD12FB5
:1031200010E00F5F1F4F0C0F1D1F84E8B82E899110
:103130008093BB00B092BC00C701B6010E94A817E3
:10314000C017D107A1F784E98093BC00DF91CF912C
:103150001F910F91FF90EF90DF90CF90BF90089557
:103160008036A0F567FD32C0E82FE695E695E69536
:10317000F0E0EE0FFF1FEA55F04FA591B4911097C4
:1031800029F1877021E030E0A90102C0440F551FEA
:103190008A95E2F7CA014FB7F89412963C911297BC
:1031A000662381F0382B282F209512963C93129796
:1031B00011963C911197232311962C9311974FBF91
:1031C000BD010895282F20953223EFCF8BE20E9476
:1031D000EB37FB012FB7F8949281411105C0809520
:1031E000892382832FBF0895892B82832FBF08955F
:1031F000FC011092260281E080934702878981605A
:10320000878B448155816681778180859185A285F0
:10321000B385840F951FA61FB71F84839583A6834C
:10322000B78381E00895FF920F931F93CF93DF93AD
:10323000EC01F88483E08F15E0F048E150E063E1B1
:1032400079E188810E9491288C0188EF98E1F8014A
:103250009383828365EA73E38C810E94C028F8011E
:10326000958B848BF68ADF91CF911F910F91FF9000
:1032700008958EE10E94EB37CF92DF92FF920F9379
:103280001F93CF93DF93EC0165EA73E38C810E9477
:10329000C0286C01F8840F2D10E0A8014D5F5F4F2E
:1032A0006CE379E188810E949128FC01D182C0827F
:1032B000F2826C857D85A8010396DF91CF911F91E5
:1032C0000F91FF90DF90CF900C949E3A8BE10E947B
:1032D000EB376F927F928F929F92AF92BF92CF9275
:1032E000DF92EF92FF920F931F93CF93DF934C01E6
:1032F000E62E142F6901DC0115967C901597872D19
:10330000867009F451C071FC39C0F401908181814B
:103310009CBD8DBDF72DF1706F2E70FCC8C0EE20E6
:1033200009F49CC08FEF810F112351F0F6019081B9
:103330009EBD0DB407FEFDCF9EB591938150B8F7A9
:10334000662091F1072D069506950695402F40952C
:103350004170D40112966D917D918C91DF91CF9146
:103360001F910F91FF90EF90DF90CF90BF90AF90A3
:103370009F908F907F906F900C94E918ED91FC9145
:10338000418542706681778180850E94E918B72D5A
:10339000B1706B2E70FC17C0D401CD91DC91AA24C2
:1033A000AA94A10E111126C0DF91CF911F910F9108
:1033B000FF90EF90DF90CF90BF90AF909F908F9055
:1033C0007F906F900895072D069506950695402FDE
:1033D0004170F4016281738184810E94E918D401F3
:1033E000CD91DC91AA24AA94A10E112309F4AECFA9
:1033F00066246394B12C8FEFA81AB80AAC0CBD1CDC
:10340000D601FC9008E010E0898580FF35C0EE8190
:10341000FF81888580834F2D40786B817C818D81F1
:103420000E94E918FF0CEE81FF8188858083110FCF
:10343000E881F98190818A81892391E009F490E003
:10344000192B015009F7EE2011F0F6011083FFEF60
:10345000CF1ADF0AAC14BD0499F672CFF6019601BB
:10346000210F311D2E173F0709F46ACF81918EBDC0
:103470000DB407FEFDCFF6CF4F2D40786B817C81D8
:103480008D810E94E918FF0CEE81FF818885808381
:10349000110FE881F98190818A81892391E009F4F3
:1034A00090E0192BEE81FF8188858083CACF73FA63
:1034B000442740F9F4016281738184810E94E918F4
:1034C000662463942CCFCF93DF93EC0165EA73E31A
:1034D00088810E94C028288539854C8160E0DF9171
:1034E000CF910C946919FF920F931F93CF93DF93A1
:1034F000EC01188165EA73E3812F0E94C0280C81DA
:10350000F884C9852F2D3C2F402F61E00E94691956
:10351000CF93FF921F920F931F921F9381ED90E123
:103520009F938F930E94C0318DB79EB708960FB6B8
:10353000F8949EBF0FBE8DBFDF91CF911F910F9169
:10354000FF900895CF93DF93EC016A8D662309F411
:1035500053C0FC0150E031E020E0A38DB48D4C91CC
:10356000958D942309F0532B2F5F330F3396261339
:10357000F4CF2C85922F952729F08D85852780956E
:103580009823D9F4888D5D8787FD03C0815070F141
:10359000888F4C815D816E817F8188859985AA8520
:1035A000BB85840F951FA61FB71F8C839D83AE8399
:1035B000BF8381E0DF91CF910895982F90952923C3
:1035C0008523822B8C879E859830E0F621E0290F99
:1035D0002E87FE01E90FF11D87871092260281E0F8
:1035E000809348028FEF888F5D87D3CF1092260299
:1035F00091E090934802CCCF50E0BBCFAF92BF9206
:10360000DF92EF92FF920F931F93CF93DF93FC0112
:10361000A485B585968547855089E18822893389B7
:10362000F488A588B6887789008D118DD28C808525
:1036300086279C9384FD20C085FD22C086FD24C082
:1036400087FD26C09C93862F8295807F8087682780
:103650009C9364FD2AC065FD25C066FD1CC067FD06
:103660001EC09C93DF91CF911F910F91FF90EF901F
:10367000DF90BF90AF900895EA01E88285FFDECF2A
:10368000E901F88286FFDCCFE501788387FFDACF96
:10369000E801D882D7CFF501708367FFE2CFE80158
:1036A000D882DFCFE901F882D8CFFA01E082D3CF08
:1036B0000F931F93CF93DF938C0164E87BE1DC01D0
:1036C0008C910E94C028FC01D80114969C91828D97
:1036D0009817B8F4292F30E0E901CC0FDD1F2C0F2B
:1036E0003D1FEF01C20FD31FF801648580850E9442
:1036F000B0186B8F7C8F8D8FDF91CF911F910F91C1
:10370000089585E20E94EB37CF93FC01C481C93054
:10371000B8F44C2F50E09A01220F331F420F531F71
:10372000455E5F4F64E87BE1FC0180810E94912847
:10373000FC01C28F22EA3AE133832283CF910895BC
:1037400086E20E94EB375F926F927F928F929F92F8
:10375000AF92BF92CF92DF92EF92FF920F931F939F
:10376000CF93DF938C01FC01C080D180E280F38095
:1037700084809580A680B78066246A94660E66234E
:1037800001F1EA01712CFFEF6F1A7F0A640E751EBA
:1037900059900E945A26DC01CB018C199D09AE0973
:1037A000BF0988159905AA05BB0598F3652DC801C1
:1037B0000E94FE1A0E945A266B017C01C615D7058D
:1037C00039F7F801C082D182E282F382DF91CF9192
:1037D0001F910F91FF90EF90DF90CF90BF90AF902F
:1037E0009F908F907F906F905F9008950F931F939D
:1037F000CF93DF93EC016EE27CE188810E94C028C8
:103800008C01FC0161857285838541E00E94E91885
:10381000488559856C81C801DF91CF911F910F9127
:103820000C94A31B0F931F93CF93DF93EC016EE2D5
:103830007CE188810E94C0288C01FC016185728531
:10384000838540E00E94E918488559856C81C8014C
:10385000DF91CF911F910F910C94A31BCF92DF9218
:10386000EF92FF920F931F93CF93DF93EC014BE105
:1038700050E06EE27CE188810E9491288C0160E03A
:103880008C810E940825F80161877287838760E038
:1038900088850E940825F80164877587868760E01F
:1038A0008C850E940825F8016787708B818B60E00A
:1038B00088890E940825F801628B738B848B60E0F5
:1038C0008C890E940825F801658B768B878B60E0D8
:1038D000888D0E940825F801608F718F828FF8947F
:1038E0000E945A266B017C0160E0C8010E94FE1A0A
:1038F0000E945A267894DC01CB018C199D09AE09EF
:10390000BF09CC8CDD8CEE8CFF8C8C159D05AE0533
:10391000BF0548F4C81AD90AEA0AFB0AF801C482AA
:10392000D582E682F782DF91CF911F910F91FF90B0
:10393000EF90DF90CF9008954F925F926F927F92B9
:103940008F929F92AF92BF92CF92DF92EF92FF92AF
:103950000F931F93CF93DF938C01562E3A01FC01F6
:1039600080809180A280B380C480D580E680F7807B
:10397000EA012196FA014080642D607F0E94642F45
:103980000E945A26DC01CB0188199909AA09BB09B2
:103990008C159D05AE05BF0598F3642D6295607F7B
:1039A000C8010E94642F0E945A266B017C01F80115
:1039B00080849184A284B384F1E05F1639F15A9433
:1039C0005A94852D90E00296680E791E5990652DC7
:1039D000607FC8010E94642F0E945A26DC01CB013F
:1039E0008C199D09AE09BF0988159905AA05BB0563
:1039F00098F3652D6295607FC8010E94642F0E9434
:103A00005A266B017C01C615D70501F7F801C08263
:103A1000D182E282F382DF91CF911F910F91FF90CB
:103A2000EF90DF90CF90BF90AF909F908F907F905E
:103A30006F905F904F900895CF92DF92EF92FF9238
:103A4000CF93DF93FC01A085B18582858C93968509
:103A500081E089278687C82FC170C688D788E08C07
:103A6000F18C97859F5FD1899D1708F05FC0892FE2
:103A7000869586958695DF01A80FB11D5A962C91E3
:103A800030E0892F877002C0359527958A95E2F737
:103A90002170B701A601C217A9F033C0892F8695FE
:103AA00086958695DF01A80FB11D5A962C9130E0BE
:103AB000892F877002C0359527958A95E2F7217086
:103AC000C2131FC04C0D5D1D6E1D7F1D9F5F9D1796
:103AD00028F387E190E29383828384819581A68194
:103AE000B781480F591F6A1F7B1F44835583668324
:103AF000778381E0DF91CF91FF90EF90DF90CF90BF
:103B00000895978784819581A681B781480F591FB1
:103B10006A1F7B1F448355836683778381E0DF912F
:103B2000CF91FF90EF90DF90CF900895B701A6015D
:103B3000D0CFCF92DF92EF92FF920F931F93CF934C
:103B4000DF93EC01E885F9858A8580830E945A26F7
:103B50003E8521E023272E872F852F5F2F87213059
:103B600009F45CC02530E0F40C811D812E813F8179
:103B70004A895B896C897D89DB01CA01800F911FAD
:103B8000A21FB31F8C839D83AE83BF8381E0DF912F
:103B9000CF911F910F91FF90EF90DF90CF900895FC
:103BA000CC80DD80EE80FF80AB01BC014C195D094B
:103BB0006E097F098E899F89A88DB98D481B590B85
:103BC0006A0B7B0BDB01CA010296A11DB11DB7FD7B
:103BD00034C0B595A79597958795B595A795979571
:103BE00087950A891B892C893D89800F911FA21F07
:103BF000B31F8E8B9F8BA88FB98F2CE13DE13B8348
:103C00002A834C0D5D1D6E1D7F1D840F951FA61F01
:103C1000B71F8C839D83AE83BF83B8CF0C811D817A
:103C20002E813F81AB01BC01401B510B620B730B1A
:103C30004E8B5F8B688F798F9BCFDB01CA01059616
:103C4000A11DB11DC6CFEF92FF920F931F93CF938B
:103C5000DF937C0164EC7EE1FC0180810E94C0283E
:103C6000EC011E8511FF07C0DF91CF911F910F91CD
:103C7000FF90EF900895F701048160857185F484C9
:103C80000B3008F045C0FAE0FF1508F441C0402FA2
:103C900050E04A960E949E3A1F86117312601E875A
:103CA000802F880F880F880F898BFF0CFF0CFF0C6B
:103CB000F88A002349F08A8D8F738A3229F489E9C2
:103CC0009DE19B838A830CC08A899B89AC89BD89CD
:103CD0008E8B9F8BA88FB98F8CE19DE19B838A830C
:103CE000F8940E945A26DC01CB018058934FAF4FC5
:103CF000BF4F8C839D83AE83BF83CE010E948635E8
:103D00007894DF91CF911F910F91FF90EF900895DC
:103D100087E20E94EB370F931F93CF93DF938C01C1
:103D200064E87BE1DC018C910E94C028EC01D801A1
:103D30001496EC918F898E0F8F8BF8948E85E817EF
:103D4000D0F48E1BF0E03F96EC0FFD1FDE011F96B6
:103D50002FEF280F30E0205F3F4F2C0F3D1F919138
:103D60009D93A217B307D9F78E877894DF91CF91EF
:103D70001F910F9108951E868EEF888F7894DF91A2
:103D8000CF911F910F9108957F928F929F92AF9242
:103D9000BF92CF92DF92EF92FF920F931F93CF9338
:103DA000DF93EC0144E250E064EC7EE188810E9404
:103DB00091288C0178848C809D80AE80BF80CC84DB
:103DC000DD84EE84FF8461E0711001C060E0882D25
:103DD0000E94B018F80163877487858761E08C2D95
:103DE0000E940825F80160877187828788899989F0
:103DF000AA89BB89828B938BA48BB58B711018C059
:103E000091E08C149D04AE04BF04C1F080E0892BC6
:103E1000F8018687DF91CF911F910F91FF90EF906E
:103E2000DF90CF90BF90AF909F908F907F9008953C
:103E300091E18C149D04AE04BF0441F780E2E7CF0A
:103E40000F931F93CF93DF938C0164E87BE1FC0118
:103E500080810E94C028EC010E943435F8018481E1
:103E60009581A681B7818C839D83AE83BF83408576
:103E7000518562857385488759876A877B878089E2
:103E80008D878C871E861F8A8EEF888F8485898F09
:103E900087FD10C0452B462B472B29F4DF91CF918E
:103EA0001F910F910895CE01DF91CF911F910F9136
:103EB0000C94863584E20E94EB37CF93DF93EC01BC
:103EC0008E8585FD0DC0688579858A8541E00E94D3
:103ED000E9188E85807381608E87DF91CF91089578
:103EE000E885F9858A852FB7F8949281982B92837B
:103EF0009181892B81832FBF8E85807381608E870E
:103F0000DF91CF910895CF93DF93FC01A385B48512
:103F10005C918785982F977021E030E001C0220FD7
:103F20009A95EAF7982F969596959695DF01A90FA1
:103F3000B11D5A969C915A9745854523E1F0292B4E
:103F40005A962C938F5F90898917E8F4878744816C
:103F500055816681778186899789A08DB18D840F7F
:103F6000951FA61FB71F84839583A683B78381E01F
:103F7000DF91CF910895209529235A962C938F5F36
:103F80009089891718F3EF01CF010E945D1F8E857C
:103F900088608E871092260281E08093490280E03B
:103FA000DF91CF910895CF93DF93FC01A385B48572
:103FB0009C9185858923E9F086858460868787853D
:103FC00091E0980F9787803408F544815581668188
:103FD000778186899789A08DB18D840F951FA61F43
:103FE000B71F84839583A683B78381E0DF91CF9148
:103FF0000895868582FFE3CF178683E89FE1938348
:104000008283CF01DF91CF910C94831FEF01108A3F
:10401000CF010E945D1F8E8588608E8710922602D8
:1040200081E08093490280E0DF91CF9108950F9362
:104030001F93CF93FC01C089CC23E9F1868585FDD0
:1040400023C0178683ED9FE19383828386899789B6
:10405000A08DB18D880F991FAA1FBB1F880F991FB4
:10406000AA1FBB1F4481558166817781840F951FEC
:10407000A61FB71F84839583A683B783C1E08C2FC7
:10408000CF911F910F910895A385B48595852FB782
:10409000F89484FF21C012968C911297892B9095E9
:1040A00012968C93129711968C91119798231196D2
:1040B0009C932FBFC6CF8C010E945D1FF80186859F
:1040C000886086871092260281E0809349028C2FB7
:1040D000CF911F910F91089512968C911297909500
:1040E0008923DECF0F931F93CF93DF93FC01A18928
:1040F000B2898D919C911197928B818B16968D919F
:104100009C911797C085D185228521113FC02FB77B
:10411000F894AC015527598348832FBF20914A0258
:1041200030914B0211963C932E93B0934B02A09387
:104130004A02A189B289109759F5278530898217DB
:10414000930741F083859485A585B6850097A105E1
:10415000B10531F480E0DF91CF911F910F91089567
:104160004481558166817781840F951FA61FB71FF3
:1041700084839583A683B78387EF90E293838283BA
:1041800081E0DF91CF911F910F9108958883C6CF71
:1041900012964D915D916D917C911597278530898F
:1041A0008217930741F083859485A585B68500978E
:1041B000A105B10551F4448355836683778381E07B
:1041C000DF91CF911F910F91089504811581268170
:1041D0003781800F911FA21FB31F2B2F84179507C4
:1041E000A607270B27FFE7CF80E20E94EB3781E28B
:1041F0000E94EB372F923F924F925F926F927F9285
:104200008F929F92AF92BF92CF92DF92EF92FF92E6
:104210000F931F93CF93DF9300D01F921F92CDB7C0
:10422000DEB77C012DB73EB73D832C836AED76E186
:10423000DC018C910E94C0289B838A83F701F48162
:10424000F983D70118966D907C9019971C968D91E3
:104250009D910D90BC91A02D80FD6BC01C012D0186
:104260005694479437942794F701E088F188C22C3C
:10427000D12CF9810F2F10E0C8018C0D9D1D2DB799
:104280003EB7281B390B0FB6F8943EBF0FBE2DBFAB
:104290008DB79EB701965C01A801B3010E949E3ABA
:1042A0004501800E911E8401222DA3016981AA81FE
:1042B000BB818C910E94DB17C114D10499F0CE0C04
:1042C000DF1CF4019601D7018D917D0180959081CD
:1042D00089238083D9019D919D01892B8193CE14DF
:1042E000DF0489F76981620DA501EA81FB81808184
:1042F0000E946518EC81FD810FB6F894FEBF0FBED9
:10430000EDBF0F900F900F900F900F90DF91CF9116
:104310001F910F91FF90EF90DF90CF90BF90AF90E3
:104320009F908F907F906F905F904F903F902F90D5
:1043300008958FE10E94EB371F93CF93DF93EC0139
:10434000162FAC89BD891097B9F01296ED91FC91AA
:1043500013978D919C9111979D8B8C8B11961C922C
:104360001E9213961C921E921297612FCD011995E1
:10437000AC89BD89109749F71092260281E080939D
:104380004C02DF91CF911F910895FC0138979689D7
:1043900090FF08C0608D678B9A7F9460968BCF01E9
:1043A0000E949C2180E00895FC0186898460868BB0
:1043B0001092260281E080934C02448155816681EF
:1043C000778180899189A289B389840F951FA61F5F
:1043D000B71F84839583A683B78381E00895FC018A
:1043E000A085B1859C9182858923D1F0818D8095AE
:1043F0008170C9F4838D815031F1838F448155815F
:104400006681778187859089A189B289840F951FFC
:10441000A61FB71F84839583A683B78381E0089581
:10442000818D817039F38FE19AE29383828383894E
:104430009489A589B68984839583A683B783828D61
:10444000838F81E00895A789B08D56969C915697E9
:10445000892F817090FFE3CF648D57966C935797A7
:104460009A7F946056969C935697CD010E949C210A
:1044700080E00895FC0180917A0086FF0EC084815F
:104480009581A681B7818853984FAF4FBF4F8483E2
:104490009583A683B78381E00895828D9091090268
:1044A000981781F09F3F59F780930902982F9870D1
:1044B00090937B008770806480937C0087ED80936D
:1044C0007A00DDCF8FEF8093090220917800309140
:1044D0007900858D968D891780F544895589240F3B
:1044E000351F8F5F358B248B858F891760F1868907
:1044F000978928173907C8F1808D918D8217930706
:10450000A0F1138E1092260281E080934D02408923
:1045100051896289738980859185A285B385840FCD
:10452000951FA61FB71F808B918BA28BB38B8483A3
:104530009583A683B78381E0089581E0358B248B32
:10454000858F8917A0F6448155816681778184859E
:104550009585A685B785840F951FA61FB71F8483F1
:104560009583A683B78381E00895838D8F5F838FC2
:10457000948D891738F2809127028111C2CF8AE188
:104580000E94EB37EF92FF921F93CF93DF937C0152
:10459000FC01108169E373E2812F0E94C028EC01C5
:1045A000F8948E8980FF09C0F70164816F8B8A7F40
:1045B00084608E8BCE010E949C21CE010E943435F6
:1045C000CE0108960E9434351E8A8F8978941F92F6
:1045D0001F921F921F921F928F931F921F921F92E2
:1045E0001F938BED90E19F938F930E94C0318DB705
:1045F0009EB70C960FB6F8949EBF0FBE8DBFDF918D
:10460000CF911F91FF90EF900895CF93FC01C0814F
:104610006FEC73E28C2F0E94C028FC01F894818D0E
:1046200033894489558966897894A085B1852C9110
:104630009285922321E009F420E01F922F936F933B
:104640005F934F933F93869581701F928F931F9234
:10465000CF9380EE90E19F938F930E94C0318DB7EE
:104660009EB70C960FB6F8949EBF0FBE8DBFCF912C
:10467000089549E150E069E373E2FC0180810E9402
:10468000912824ED31E2FC013383228325EC31E2D1
:10469000338722870895EF92FF920F931F93CF9352
:1046A000DF938C0169E373E2FC0180810E94C028E2
:1046B000EC01F8948E8980FF13C07E01F8E0EF0EC4
:1046C000F11CC7010E943435F80184819581A681CF
:1046D000B7818C879D87AE87BF87C7010E948635CB
:1046E0007894DF91CF911F910F91FF90EF900895F3
:1046F0000F931F93CF93DF938C016FEC73E2FC0158
:1047000080810E94C028EC010E943435F801848128
:104710009581A681B7818C839D83AE83BF8380857D
:104720009185A285B3858F87988BA98BBA8B848559
:104730008A8F882361F1F8014089518962897389E0
:104740004B875C876D877E872FE13AE23B832A8324
:104750008B8F84899589A689B789892B8A2B8B2B86
:10476000A1F482E0898F69E373E2F801808D0E94F1
:10477000C028988F8F8BF801848D8C8FCE01DF91AC
:10478000CF911F910F910C94863583E0EBCF188E5B
:104790001F8A198EDF91CF911F910F9108950F936A
:1047A0001F93CF93DF93EC014DE150E06FEC73E288
:1047B00088810E9491288C0168858C810E94B018A4
:1047C000F801608771878287DF91CF911F910F91E8
:1047D0000895CF93DF93EC010E943435CE01089603
:1047E0000E943435EC89FD89309751F090818181A8
:1047F0001382128211821082E92FF82F3097B1F7BD
:104800001D8A1C8A188E1F8A1E8ADF91CF910895F7
:104810000F931F93CF93DF938C0169E373E2FC0145
:1048200080810E94C028EC01F8940E94E92381E075
:104830008E8BF80184819581A681B7818C839D83BD
:10484000AE83BF8380859185A285B385888B998B44
:10485000AA8BBB8B892B8A2B8B2B19F0CE010E9444
:104860008635F8018485888F7894DF91CF911F91E8
:104870000F910895B0990FC080914F02909150020E
:104880000196109205021092040290930702809301
:10489000060281E0089581E086BB80914F029091ED
:1048A000500201969093500280934F0220E030E82E
:1048B000309305022093040290930702809306022E
:1048C00081E00895CF93DF93FC0184819581A681D7
:1048D000B7814489558966897789C58DD68D388198
:1048E000C42FC170278D232331E009F430E0C317B2
:1048F00061F04F5F5F4F6F4F7F4F448B558B668BDF
:10490000778B808F918FA28FB38F40895189628975
:104910007389272F481759076A072B0B27FF18C0E1
:10492000248D2160248F4485558566857785840F85
:10493000951FA61FB71F808B918BA28BB38B1092F4
:10494000260281E080934E0284819581A681B78101
:104950004085518562857385840F951FA61FB71FFB
:1049600084839583A683B78381E0DF91CF910895F7
:104970000F931F93CF93DF938C016AEE74E2FC01D7
:1049800080810E94C028EC010E943435F8018481A6
:104990009581A681B7818C839D83AE83BF8340853B
:1049A000518562857385488759876A877B874485E7
:1049B0005585668577854C875D876E877F87888B71
:1049C000998BAA8BBB8BCE01DF91CF911F910F9159
:1049D0000C9486350F931F93CF93DF93EC0140E245
:1049E00050E06AEE74E288810E9491288C0168850B
:1049F0008C810E94B018F801658F768F878F82E6D0
:104A000094E293838283DF91CF911F910F91089558
:104A1000803678F5E82FE695E695E695F0E0EE0F1E
:104A2000FF1FEA55F04FA591B491109711F18770CF
:104A300021E030E0A90102C0440F551F8A95E2F73A
:104A4000CA013FB7F89412962C91129761110FC0CA
:104A50004095242312962C93129711962C9111971E
:104A6000282B11962C9311973FBFBD010895242B3D
:104A7000F1CF8CE20E94EB371F920F920FB60F928C
:104A800011240BB60F92EF92FF920F931F932F9367
:104A90003F934F935F936F937F938F939F93AF93C6
:104AA000BF93CF93DF93EF93FF930DC07A01809173
:104AB0008400909185008E199F0997FD7CC07894A1
:104AC000B2999AC0F894C0912202D0912302EA814F
:104AD000FB81309709F0ADC0EA8DFB8D2C8D2083D2
:104AE0008E859F85019709F4C1C09F878E87888531
:104AF0009985AA85BB854C815D816E817F81480F38
:104B0000591F6A1F7B1F4C835D836E837F832083C5
:104B10002CA525FF0EC00C851D85012E000C220B37
:104B2000330B800F911FA21FB31F88879987AA8715
:104B3000BB87E881F9810481158126813781872F20
:104B4000401751076207830B87FDB0CF7801F093C0
:104B50002302E0932202A0912402B0912502149630
:104B60000D911D912D913C911797872F401751075B
:104B70006207830B87FFFD01DF010190F081E02DCB
:104B80000481158126813781872F401751076207DD
:104B9000830B87FFF1CFF983E883CD93DC93D09328
:104BA0002502C093240280918400909185008E1983
:104BB0009F0997FF84CF863A9F4F0CF06AC0F0920E
:104BC0008900E0928800FF91EF91DF91CF91BF9132
:104BD000AF919F918F917F916F915F914F913F9195
:104BE0002F911F910F91FF90EF900F900BBE0F90A0
:104BF0000FBE0F901F901895F894809184009091AB
:104C000085009701281B390B2038314CDCF12091AD
:104C1000260227FF43C09C01205C304E30938B005E
:104C200020938A0024E026BB90938900809388001B
:104C30003ECFCE0119954C815D816E817F818111BE
:104C400078CFE881F981E480F580F0932302E09346
:104C500022028091240290912502C817D90709F0F9
:104C600026CFF0932502E093240221CFCE010E94AB
:104C7000DE2CEA8DFB8D9C8D90834C815D816E8155
:104C80007F81DDCF209127022111C1CF8AE20E94CE
:104C9000EB377894B299B0CFF89409CF9C0128549F
:104CA000344F30938B0020938A0024E026BB7C0194
:104CB000F39485CF2FB7F8946091840070918500AC
:104CC00080914F0290915002B09902C02FBF089579
:104CD0002FBF7F3FE1F30196089578940E94043638
:104CE0002FEF260F6623C1F0FC018FEF9FEF31916C
:104CF0008327082E8295807F8025092E982F829504
:104D00008F700826869598278927880F880F880F27
:104D10008025215060F708958FEF9FEF08950F933E
:104D20001F93FC01A489B58986898C9393A181E0A6
:104D3000892783A3448155816681778180FF12C0D2
:104D40000085118522853385400F511F621F731F17
:104D500082FD12C0448355836683778381E01F916F
:104D60000F9108950485158526853785400F511FBD
:104D7000621F731F82FFEECF008911892289338958
:104D8000872F401751076207830B87FDE3CF83EF1F
:104D900096E293838283B901A80144835583668395
:104DA000778381E01F910F9108950895FC01808120
:104DB000A481B58140855185628573859FB7F8943C
:104DC000813061F0823019F04C939FBF08954D936C
:104DD0005D936D937C9313979FBF089511965C9399
:104DE0004E939FBF08958F929F92AF92BF92CF92A2
:104DF000DF92EF92FF921F93CF93DF93EC01EF8C42
:104E0000F8A0E114F10409F4F0C0F7018081918168
:104E100098A38F8F86809780A084B18411E081143D
:104E20009104A104B10409F4A1C06C897D898E8923
:104E3000412F0E94E91880914A0290914B02F7019C
:104E400091838083F0924B02E0924A028114910494
:104E5000A104B104E9F08B8D9C8DAD8DBE8D8816BB
:104E60009906AA06BB06A0F44F89588D698D7A8DE4
:104E7000411551056105710509F45BC08C819D8167
:104E8000AE81BF81480F591F6A1F7B1F166022C069
:104E90008BA131E081149104A104B10409F068C030
:104EA00084FB992790F921E09227391709F443C030
:104EB0004F89588D698D7A8D4115510561057105B0
:104EC000D1F18C819D81AE81BF81480F591F6A1F2E
:104ED0007B1F1460EF8DF8A1309709F077C02BA1EC
:104EE000488B598B6A8B7B8B2071212B2BA311FF55
:104EF0005FC0880D991DAA1DBB1D12FD52C02FE871
:104F000036E23B832A838C839D83AE83BF8388866E
:104F10009986AA86BB868B8D9C8DAD8DBE8D88199A
:104F20009909AA09BB098C879D87AE87BF8781E055
:104F300011C012608BA1EF8DF8A13097D9F4188AB7
:104F4000198A1A8A1B8A8071812B8BA3812F827008
:104F500011FD34C0DF91CF911F91FF90EF90DF9052
:104F6000CF90BF90AF909F908F90089510E05DCF4D
:104F700030E096CF4281538164817581488B598B93
:104F80006A8B7B8B8071912F9460892B8BA311FF8F
:104F90000FC08C819D81AE81BF81880D991DAA1D96
:104FA000BB1D2B2F84179507A607270B27FDA7CF1F
:104FB0004C835D836E837F8381E0CCCF40E050E003
:104FC000BA018C819D81AE81BF8193CFC280D38095
:104FD000E480F580872F4C155D056E058F0987FDF0
:104FE00007C08BA1B701A601C9CF85E10E94EB37AD
:104FF00083E10E94EB37FC0185818F9384818F933D
:1050000080811F928F938FEE90E19F938F930E94E8
:10501000C0310F900F900F900F900F900F90089548
:10502000DC012C911496ED91FC9115973FB7F89403
:105030002130E9F02230B1F0808190E0A0E0B0E0D2
:105040003FBFBF93AF939F938F938AEE90E19F935F
:105050008F930E94C0310F900F900F900F900F9080
:105060000F90089580819181A281B381E9CF8081E1
:105070009181A0E0B0E0E4CFCF92DF92EF92FF9277
:10508000FC0140815181628173812481E2EAFFE069
:1050900085919591A591B491481759076A077B07A7
:1050A00070F56A017B01C20ED11CE11CF11C8C154C
:1050B0009D05AE05BF0500F5841B90E09A01225CBA
:1050C0003A4F3F932F939F938F937F936F935F9369
:1050D0004F9388E091E19F938F930E94C0318DB7E9
:1050E0009EB70A960FB6F8949EBF0FBE8DBFFF9075
:1050F000EF90DF90CF900895822F90E0DFCF80E097
:1051000090E0DCCF80912702882329F0823011F0D3
:1051100010922702089582E00E94EB378EE00E94F1
:10512000EB37CF93DF9390913702891730F5C82F73
:10513000D0E0CC0FDD1FCC0FDD1FE0913802F091E5
:105140003902EC0FFD1F80819181892BB1F4809190
:105150003F0290914002892B81F471836083CA01E0
:105160000E949D312091380230913902C20FD31F25
:105170009B838A83DF91CF9108958BE00E94EB3768
:1051800090913702891788F4E0913802F091390242
:1051900094E0899FE00DF11D112480819181861793
:1051A000970719F48281938108958CE00E94EB3770
:1051B000CF92DF92EF92FF92CF93DF93C0913F02A5
:1051C000D09140022097B9F121976E01E12CF12C8A
:1051D000A0913E02B0E02097D9F020E030E040E01E
:1051E00050E0BA0180913C0290913D02FC01E20F37
:1051F000F31F4F5F5F4F6F4F7F4F2A0F3B1F820F91
:10520000931F918380834C155D056E057F0550F3D8
:1052100080913C0290913D02CA9FF001CB9FF00D1E
:10522000DA9FF00D1124E80FF91F1182108290937C
:105230004B0280934A02DF91CF91FF90EF90DF9075
:10524000CF900895FC0113821282118210826F3F69
:10525000710509F07CF480913F0290914002892B06
:1052600049F480913E0290E08617970714F460930A
:105270003E0208950E948E282FB7F89480914A022A
:1052800090914B02009749F0FC014081518150936D
:105290004B0240934A022FBF08958FE00E94EB37E4
:1052A000CF92DF92EF92FF921F93CF93DF936A0129
:1052B0007B016EEB7FE0FB019491981749F0675FEB
:1052C0007F4FF0E16E347F07B1F784E30E94EB3744
:1052D000FB013896949191FF1AC030EAC3163FE55E
:1052E000D306E104F10408F483C0C0E8CC16CEE78D
:1052F000DC06C1E0EC06F10408F090C0D0E4CD1665
:10530000DFEBDD06E104F104C8F414E022C0F8EBA1
:10531000CF16F7E4DF06E104F10490F0A0ECCA1622
:10532000AEE3DA06A1E0EA06F10408F475C0C114A0
:10533000BBEFDB06B4E0EB06F10438F315E009C07F
:1053400037EFC31638E0D306E104F10408F05FC07C
:1053500011E0FB013396A591B491FB013596C591FF
:10536000D491FB0137963491E82FE695E695E695C2
:10537000F0E0EE0FFF1FEA55F04F45915491877012
:10538000E1E0F0E07F0101C0EE0C8A95EAF7FB0155
:105390003196C590D490892F8170A038B10509F459
:1053A0004BC0EFB7F8949881977011F0191341C072
:1053B000188381112EC09FB7F894622F70E0E60128
:1053C000798368839FBF9C913160392B3C93DA01CC
:1053D00011969C911197E92A1196EC92EFBFB601B4
:1053E000DF91CF911F91FF90EF90DF90CF900895C4
:1053F000A8EDCA16A7E2DA06E104F10468F4B7EFF3
:10540000CB16B8E0DB06E104F10408F4A1CF12E00A
:10541000A0CFE6012883D7CF13E09BCFC114EBEFD9
:10542000DE06E4E0EE06F10410F416E092CF17E099
:1054300090CF82E30E94EB3783E30E94EB370F9318
:105440001F93FC01A085B1859C9104811581268163
:1054500037814385548565857685400F511F621FCE
:10546000731F8285892361F0818D8095817059F049
:10547000448355836683778381E01F910F9108955C
:10548000818D8170A9F7438B548B658B768B8FEE62
:1054900091E293838283CF011F910F910C94EF21AE
:1054A000CF93DF93EC0168E87CE288810E94C028FA
:1054B000FC018C819D81AE81BF81892B8A2B8B2B36
:1054C00051F420E0F89494A59D7F922B94A77894B2
:1054D000DF91CF91089522E0F5CF0F931F93CF93E3
:1054E000DF938C01EC01A897CE010E9434351C8219
:1054F0001D821E821F821A8A1B8A1C8A1D8A88A10D
:1055000099A1AAA1BBA12CA54E855F85688979893F
:1055100024FD04C07695679557954795841B950B98
:10552000A60BB70BB7FD40C0B095A095909581959F
:105530009F4FAF4FBF4F88A399A3AAA3BBA31E86BB
:105540001F86188A198A247128602CA76D8D7E8D7C
:105550008F8D40E00E94E9184CA544706A8D7B8DC8
:105560008C8D0E94E918D8011497ED91FC91119748
:105570003097A9F040914A0290914B0201C0F90185
:105580002081318140839183F0934B02E0934A0262
:105590004E2F9F2F2115310591F71D921C92DF91FF
:1055A000CF911F910F910895B095A09590958195F9
:1055B0009F4FAF4FBF4FB8CF0F931F93CF93DF9342
:1055C0008C0168E87CE2FC0180810E94C028EC012B
:1055D00069E373E2F80184810E94C028BE01685D1E
:1055E0007F4F4FB7F8942AA53BA5232B89F42DE6CE
:1055F0003AE23BA72AA7FC012489358939A728A7C5
:10560000758B648B4FBFDF91CF911F910F910895E0
:1056100089E10E94EB37CF93DF93EC0168E87CE2ED
:1056200088810E94C028FC018C819D81AE81BF8150
:10563000F8944685578560897189452B462B472B01
:1056400079F484839583A683B783828B938BA48B11
:10565000B58B84A5877F84A77894DF91CF91089537
:1056600086E10E94EB37CF93FC01C08168E87CE2C1
:105670008C2F0E94C028FC01F89480A191A1A2A1C6
:10568000B3A124A5468557856089718924FD04C08E
:105690007695679557954795841B950BA60BB70B89
:1056A000B7FF07C0B095A095909581959F4FAF4FDC
:1056B000BF4F7894B054BF93AF939F938F931F9233
:1056C000CF9385EE90E19F938F930E94C0318DB769
:1056D0009EB708960FB6F8949EBF0FBE8DBFCF91B0
:1056E00008954F925F926F927F92BF92CF92DF9216
:1056F000EF92FF920F931F93CF93DF93FC01B08043
:1057000066E47CE28B2D0E94C028EC014D805E8017
:105710006F807884C984DA84EB84FC840E945A26E2
:10572000DC01CB0184199509A609B7098C159D05E3
:10573000AE05BF0568F40E945A26DC01CB0184192E
:105740009509A609B7098C159D05AE05BF0598F307
:10575000CD84DE84688179818A81A0918400B091B2
:1057600085000B811C819E01215F3F4F7901C20E94
:10577000D31ECE14DF0409F457C0F70191917F01C5
:1057800028E013C0F8944091840050918500FB01FB
:10579000808380837894FA01EA1BFB0BE017F10702
:1057A000D8F4990FDA01215021F397FFEBCFF89449
:1057B0004091840050918500FB0180837894FA0128
:1057C000EA1BFB0BE017F10738F4990FF894FB0183
:1057D00080837894DA01E7CF40E00E94E9180E94C4
:1057E0005A266D837E838F83988780E01F928F93E4
:1057F0001F92BF9285E990E19F938F930E94C031E1
:105800000F900F900F900F900F900F90DF91CF910E
:105810001F910F91FF90EF90DF90CF90BF907F90FE
:105820006F905F904F9008950E945A266D837E83FB
:105830008F83988781E0DACF0F931F93CF93DF9305
:10584000EC0166E47CE288810E94C0280C811D8105
:105850002E813F8148856C857D8517FD14C050E001
:10586000DA01A00FB11FEC01ED85FE85EA17FB07F9
:1058700050F0015F1F4F800F911FDF91CF911F915B
:105880000F910C949E3A88E20E94EB376F927F92C0
:105890008F92CF92DF92EF92FF92CF93DF93EC0142
:1058A00060E08C810E9408253B01882EC884D98441
:1058B000EA84FB84D7FC24C0A601415F5F4F66E405
:1058C0007CE288810E949128FC0160827182828240
:1058D000D686C5868C859D8594838383888999899E
:1058E000AA89BB8981879287A387B487DF91CF91EB
:1058F000FF90EF90DF90CF908F907F906F90089502
:1059000089E20E94EB37FC01648180810C940825B8
:105910000F931F93CF93DF938C014DE250E068E823
:105920007CE2FC0180810E949128EC01F8018485D1
:1059300018160CF041C064E06CA7F80184810E9445
:1059400008256A8F7B8F8C8F60E0F80180850E942C
:1059500008256D8F7E8F8F8F80E090E0A0E0B0EC07
:1059600088A399A3AAA3BBA3F80180899189A289DE
:10597000B3898E8B9F8BA88FB98F6BE070E0CE01BF
:1059800084960E9422298E899F89A88DB98D899736
:10599000A105B10548F08BE19EE29B838A83DF91EC
:1059A000CF911F910F9108958CA580618CA7DF91F5
:1059B000CF911F910F91089560E0BECFCF92DF92FB
:1059C000EF92FF92CF93DF93FC01A4A1B5A11097B2
:1059D00061F416861786108A118A80E0DF91CF91D4
:1059E000FF90EF90DF90CF9008958D919C9111974B
:1059F00095A384A316968D919C911797958784877C
:105A00001296CD90DD90ED90FC901597AC01092E8B
:105A1000000C660B770B4C0D5D1D6E1D7F1D4087C6
:105A200051876287738724A524FD43C04289538927
:105A300064897589C40ED51EE61EF71EC28AD38AF4
:105A4000E48AF58AC482D582E682F78218968D911F
:105A50009C911997AC0160E070E0440F551F661FE0
:105A6000771F46875787608B718B1A962C911A97F0
:105A700020FD3FC040A151A162A173A1480F591F51
:105A8000611D711D40A351A362A373A380914A02BB
:105A900090914B0211969C938E93B0934B02A093DE
:105AA0004A0281E0DF91CF91FF90EF90DF90CF909D
:105AB00008954481558166817781C40ED51EE61E06
:105AC000F71EC482D582E682F782892B31F12062EB
:105AD00024A718968D919C911997AC0160E070E015
:105AE00046875787608B718B1A962C911A9720FFE7
:105AF000C1CFAC0160E070E0C0A0D1A0E2A0F3A0F3
:105B00004C195D096E097F0940A351A362A373A3D9
:105B1000C58DD68D878D8883B9CF2F7DD9CF0F9333
:105B20001F93CF93DF938C0168E87CE2DC018C91BA
:105B30000E94C028EC010E943C29FC01D801149667
:105B40004D915D916D917C9117974283538364834E
:105B5000758318968D919C91199791878087892BD1
:105B600009F466C0D8011C968D919C911D9797836E
:105B700086831286F8948CA5282F217081FB9927A3
:105B800090F9291729F091E08927928591609287F1
:105B90004E855F8568897989452B462B472B59F5BA
:105BA00083FD19C08CA7118210828CA19DA1892B25
:105BB000A9F1AEA1BFA1ED93FC93FFA3EEA3CE018B
:105BC0000E94DE2CCE010E9486357894DF91CF9121
:105BD0001F910F91089580914A0290914B029183F9
:105BE0008083F0934B02E0934A027894DF91CF9147
:105BF0001F910F9108958CA7118210828CA19DA1F5
:105C0000892B89F0AEA1BFA1ED93FC93FFA3EEA376
:105C10007894DF91CF911F910F910895FFA3EEA388
:105C2000FDA3ECA3CCCFFFA3EEA3FDA3ECA3CDCFAC
:105C300087E10E94EB37CF92DF92EF92FF920F93B2
:105C40001F93CF93DF93EC01EA8DFB8D8C8D8083C6
:105C50000E945A260E891F89288D398D6B017C017F
:105C6000C00ED11EE21EF31E8E859F85A889B989BC
:105C70000197A109B1098E879F87A88BB98B80FFF7
:105C80000EC0CC82DD82EE82FF8281E0DF91CF9177
:105C90001F910F91FF90EF90DF90CF900895892B87
:105CA0008A2B8B2B59F1488559856A857B858A8992
:105CB0009B89AC89BD89840F951FA61FB71F8A8B4E
:105CC0009B8BAC8BBD8B0C851D85012E000C220B94
:105CD000330B400F511F621F731F488759876A8714
:105CE0007B872B2F8C159D05AE052F0927FDC9CF6E
:105CF0008C839D83AE83BF8381E0C8CFCE010E9499
:105D0000DE2C811102C080E0C1CF4C815D816E81AB
:105D10007F81972F4C155D056E059F0997FFB6CFC4
:105D20004C195D096E097F094038514C6F4F7F4F08
:105D30000CF0A7CF88E10E94EB370F931F93CF930E
:105D4000DF938C0144E450E06DE97EE2FC01808148
:105D50000E949128EC0182EF97E39B838A836AED8E
:105D600076E1F80184810E94C0289D878C87DF91AD
:105D7000CF911F910F9108954F925F926F927F92F2
:105D80008F929F92AF92BF92CF92DF92EF92FF924B
:105D90000F931F93CF93DF9300D0CDB7DEB76C0185
:105DA0006DE97EE2DC018C910E94C0287C010E949A
:105DB0005A264B015C0182E78B83D7011C96ED913B
:105DC000FC911D978E010F5F1F4F22E0AE014D5FCA
:105DD0005F4F61E080810E94DB170E945A262B01F1
:105DE0003C0129812F712983F70181898F93808953
:105DF0008F9330E0322F22278A81282BABEABAEA30
:105E00000E94273A96958795969587959F938F93AD
:105E100083891F928F9387858F9386858F934818E8
:105E200059086A087B087F926F925F924F92BF92E7
:105E3000AF929F928F92D6018C911F928F9389EA95
:105E400090E19F938F930E94C0310FB6F894DEBF0C
:105E50000FBECDBF0F900F900F90DF91CF911F918C
:105E60000F91FF90EF90DF90CF90BF90AF909F90F9
:105E70008F907F906F905F904F900895CF93DF93B6
:105E8000EC0144969F938F938B891F928F938F85FC
:105E90008F938E858F931F926F9384EA90E19F93E7
:105EA0008F930E94C0311B8A8E859F8501969F87A4
:105EB0008E878DB79EB70A960FB6F8949EBF0FBE19
:105EC0008DBFDF91CF910895CF93DF93DC011C96B6
:105ED000ED91FC911D971E969C911E971F96CD915A
:105EE000DC91509751962C9188E005C09083660F05
:105EF0009083815049F067FFF9CF288360959083A4
:105F0000660F90838150B9F7DF91CF9108950F9379
:105F10001F93CF93DF93EC0166EA7FE288810E94B2
:105F2000C0288C016AEF0E94642F6C81611105C04A
:105F3000DF91CF911F910F91089548855985C80130
:105F4000DF91CF911F910F910C949C1CCF92DF9207
:105F5000EF92FF920F931F93CF93DF938C0142E157
:105F600050E066EA7FE2FC0180810E949128EC010A
:105F700060E0F80180850E9408256C877D878E8708
:105F800060E0F80184850E9408256F87788B898BF3
:105F900061E0F80184810E94082568EFCE010E942B
:105FA000642F60E2CE010E94642FF8940E945A266A
:105FB0006B017C0160E0CE010E94642F0E945A2692
:105FC0007894688379838A839B83DC01CB018C1965
:105FD0009D09AE09BF09F801C088D188E288F3881D
:105FE0008C159D05AE05BF0540F4C81AD90AEA0A0A
:105FF000FB0ACC82DD82EE82FF82F80104891589DA
:106000002689378980179107A207B30740F4081B38
:10601000190B2A0B3B0B088719872A873B87DF91CF
:10602000CF911F910F91FF90EF90DF90CF90089547
:106030000F931F93CF93DF93EC0166EA7FE2888191
:106040000E94C0288C0168EF0E94642F6C8161114E
:1060500005C0DF91CF911F910F9108954885598513
:10606000C801DF91CF911F910F910C949C1C0F934D
:106070001F93CF93DF93EC01F8940E945A26088572
:1060800019852A853B85DC01CB01800F911FA21F5A
:10609000B31F8C839D83AE83BF83CE010E94863560
:1060A0007894DF91CF911F910F910895AF92BF9295
:1060B000CF92DF92EF92FF920F931F93CF93DF93D4
:1060C0001F92CDB7DEB77C01A62E0E94A5386C01C9
:1060D0008AEFC81681E0D80650F0D70150968D910E
:1060E0009C915197019651969C938E93509784E77B
:1060F0008983F7012389022F10E080E390E0801B61
:10610000910BC816D90640F58C2D9BEA899F812DED
:10611000112486958695982F990F890FB82EBB0C60
:10612000F1F4D70152968C9181FF0AC0C7010E94F9
:106130003435F70182898B7F828BC7010E9437300B
:106140000F90DF91CF911F910F91FF90EF90DF9013
:10615000CF90BF90AF90089580E3821BD6CF0C5EA6
:106160001F4F0E0D1F1DD7011C96ED91FC911D9721
:106170002B2DAE014F5F5F4F61E080810E94DB17E6
:10618000F70183898B0D838B8B32D8F48BEAB89E11
:10619000B12C1124B694B6944B2D50E09601ABEA85
:1061A000BAEA0E94273A969587959695879548175B
:1061B000590708F0B6CF1092260281E08093510271
:1061C000BFCF6A2DC7010E943E2FE0CF4F925F9252
:1061D0006F927F928F929F92AF92BF92CF92DF92F7
:1061E000FF920F931F93CF93DF931F921F92CDB710
:1061F000DEB76C01DC01FC906DE97EE28F2D0E9420
:10620000C0288C01F60180859185A285B385892BF4
:106210008A2B8B2B99F1C8010E943435F6018481B9
:106220009581A681B781F80184839583A683B7837E
:10623000F60180859185A285B385F80180879187D5
:10624000A287B38781E0828B118A108A178616860F
:10625000138AC8010E9486350F900F90DF91CF916D
:106260001F910F91FF90DF90CF90BF90AF909F90C4
:106270008F907F906F905F904F900895C8010E941B
:106280003435D80152961C9283E289831A820E9487
:106290005A264B015C01D8011C96ED91FC911D978B
:1062A000AE014F5F5F4F62E080810E9465180E94DF
:1062B0005A262B013C01C8010E94A538069748F0D8
:1062C0006F2DC8010E945630C8010E94A53806975C
:1062D000B8F7F8018389882339F06F2DC8010E942F
:1062E0003E2FD80153968C91F80191899F93908904
:1062F0009F931F921F921F928F9387858F938685FE
:106300008F93D301C20188199909AA09BB09BF93C8
:10631000AF939F938F93BF92AF929F928F921F9252
:10632000FF9289EA90E19F938F930E94C0310FB64C
:10633000F894DEBF0FBECDBF8FCFCF93DF93C09158
:106340003A02D0913B02AE01480F591F2DB73EB71C
:1063500021503F4F22273A952417350770F050936C
:106360003B0240933A02AC0160E070E0CE010E9433
:10637000B93ACE01DF91CF91089581E10E94EB37C8
:106380002F923F925F926F927F928F929F92AF92E5
:10639000BF92CF92DF92EF92FF920F931F93CF9312
:1063A000DF93CDB7DEB728970FB6F894DEBF0FBEE8
:1063B000CDBF809152028823C1F028960FB6F89481
:1063C000DEBF0FBECDBFDF91CF911F910F91FF9028
:1063D000EF90DF90CF90BF90AF909F908F907F9085
:1063E0006F905F903F902F90089581E080935202CC
:1063F0008E01015E1F4F2091960350909503251545
:10640000C0F4452D50E0CD8CDE8C3FEFC31AD30A8B
:10641000F60184913A01680E711CC3018136910521
:1064200054F1821B91098136910560F0109252025D
:10643000C4CF109295031092960340E050E0512C87
:1064400020E0E1CF1092950360919603561AE52C57
:10645000F12C70E06B5C7C4FA70185E393E00E9418
:10646000A73A10929603509295038091C1008062E2
:106470008093C100A7019A012B5C3C4F7901F60182
:10648000A491A63008F42BC1AA2EB12CF3E0AF1AC8
:10649000B108A20EB31EED8DFE8D32969491ED8D56
:1064A000FE8D3396C590D4902D5F3F4F3E832D8354
:1064B000ED8DFE8D8491D70112968C933601690E75
:1064C000711C78866F826F807884C614D70409F4B3
:1064D00035C18D809E80A814B90448F0F6018491DE
:1064E000853009F4BFC008F441C0883018F086E058
:1064F0000E94EB37F80120813181F5016D807E80AB
:10650000E619F709AF01FF0F660B770B49835A8332
:106510006B837C83A901330F660B770B69807A80CC
:106520008B809C80641675068606970608F4C8C0A2
:106530006D807E802FEF621A720AAD81BE814C930E
:106540001801B4E02B0E311CF801228133818A013D
:10655000B901863009F4B7C0C3010E949E3A4301D5
:10656000800E911E9E828D828101A6C0823008F429
:10657000AEC0833009F4D8C0F801408151813A019E
:10658000812C912C0E5F1F4FD401C3018096A11D59
:10659000B11D80389105A105B10508F4C2C0A40160
:1065A0009301305F4F4F5F4F211530444105510536
:1065B00008F43FC0D401C30118960097A042B1056A
:1065C00040F1A40193015C5F211531054105504163
:1065D00080F0D401C3015CE1B695A79597958795A6
:1065E0005A95D1F78068AD81BE818C931196BE8398
:1065F000AD83D401C30145E1B695A79597958795DD
:106600004A95D1F78068AD81BE818C931196BE8387
:10661000AD83D401C3013EE0B695A79597958795C4
:106620003A95D1F78068AD81BE818C931196BE8377
:10663000AD83ED81FE813196D401C30127E0B6958B
:10664000A795979587952A95D1F78068AD81BE81EA
:106650008C939F012F5F3F4F3E832D83462D4F77B5
:1066600040832AC098012E5F3F4FF801A081B1817D
:106670008D819E8101966C91662399F08A159B0508
:1066800080F4FD01319604C0A816B90609F447C08C
:106690000196AC0141505109DA016C93619161118D
:1066A000F3CFAC016D807E80461957094150D3016C
:1066B0004C939E838D8389012FEFC21AD20A03CF98
:1066C000B401A30135CFC3010E94883A48CFD80155
:1066D0006D907D908D909C900C5F1F4F55CF1A2F21
:1066E000D7011C938091080211968C936DEF610F76
:1066F000C7010E947026E10EF11CF70133979083C9
:106700003196808331968EE78083A52DA10FA093CB
:1067100095038091C10080628093C10087CEC5013E
:10672000C0CFED81FE8195CFD8014D915C913A01AA
:10673000550F880899080E5F1F4F26CF0D811E81C7
:106740000E191F0913E0100FCBCFFF920F931F9369
:10675000CF93DF938C0146E050E065EA73E3FC01E0
:1067600080810E949128EC01F801F08461E0F11031
:1067700060E0F80184810E9408256A837B838C8312
:106780008D81F11009C091E0892B8D83DF91CF912C
:106790001F910F91FF90089599E0892B8D83DF91D0
:1067A000CF911F910F91FF90089546E050E065EA68
:1067B00073E3FC0180810C9491288F929F92AF9299
:1067C000BF92FF920F931F93CF93DF93EC0165EA83
:1067D00073E388810E94C0288C01F88483E08F15C0
:1067E00008F484C0F8018581867009F07FC08C842C
:1067F0009D84AE84BF848C819D81AE81BF81892BB5
:106800008A2B8B2B09F074C0E8EAFFE0A591B491C4
:1068100011968C9180FD04C060E088E00E940825FC
:1068200060E089E00E94082560E08AE00E94082577
:1068300060E08BE00E94B01880E58CBD1DBC811427
:10684000F2E19F06FAE7AF06B10408F041C08114F7
:1068500089E098068DE3A806B10418F5E0E88E16E5
:10686000E4E89E06EEE1AE06B104C0F5F0E48F1652
:10687000F2E49F06FFE0AF06B10468F580E28816F7
:1068800081EA980687E0A806B10458F590E0E0E9AF
:106890008E16E0ED9E06E3E0AE06B10428F583E037
:1068A00002C090E080E0CF2DCC0FCC0FC065C82B8C
:1068B000F801C0839183858184608583DF91CF91C6
:1068C0001F910F91FF90BF90AF909F908F90089570
:1068D00091E080E0E8CF90E081E0E5CF91E081E0D9
:1068E000E2CF91E082E0DFCF82E0DDCF0E94661947
:1068F0008EE20E94EB37CF93DC0114969C911497A3
:1069000020E030E0C22FF901E45EFE4EE4919E17D4
:1069100041F02F5F3F4F20313105A1F78DE20E94FA
:10692000EB3787E980937A002830E8F420917E00E5
:1069300081E090E00C2E01C0880F0A94EAF7822BC8
:1069400080937E004FE150E06BE774E38C910E94EE
:106950009128FC018AE392E293838283C28F81E0D3
:10696000858FCF91089520917D003C2F377081E075
:1069700090E001C0880F3A95EAF7822B80937D0062
:10698000E1CF0F931F93CF93DF938C016BE774E3F9
:10699000FC0180810E94C028EC010E943435909156
:1069A00009028A8D981303C08FEF80930902F801C2
:1069B00084819581A681B781888B998BAA8BBB8BAB
:1069C0008C839D83AE83BF8380859185A285B385AB
:1069D0008C879D87AE87BF8784858E8F91E0980FC7
:1069E0009D8F4089518962897389488759876A8751
:1069F0007B87248935893F8B2E8B208D318D398F74
:106A0000288F948D9C8F811105C0DF91CF911F91AC
:106A10000F910895CE01DF91CF911F910F910C94AA
:106A2000863580E0089510922602EAE1F2E0848142
:106A30009581A681B781AC01BD015659674E7F4F44
:106A400044835583668377839659A74EBF478093C7
:106A5000160290931702A0931802B093190281E0D6
:106A6000089584E00E94EB370F931F934FB7F8947B
:106A7000E0912202F0912302E817F90729F42AC0D5
:106A80008217930789F0F9012081318121153105A1
:106A9000B9F720912402309125028217930781F0E3
:106AA0004FBF1F910F910895DC012D913C913183CF
:106AB000208320912402309125028217930781F7C9
:106AC0008AE192E090932502809324024FBF1F91A8
:106AD0000F910895DC0114960D911D912D913C911B
:106AE000179700930E0210930F0220931002309319
:106AF00011022D913C9130930B0220930A022AE05F
:106B000032E03093230220932202C3CFAF92BF9290
:106B1000CF92DF92EF92FF921F93CF93DF93DC012E
:106B20001496CD90DD90ED90FC9017971FB7F894D8
:106B3000C0912202D09123024C815D816E817F81C0
:106B40008F2DC416D506E606870B87FD1FC0FE01F4
:106B50000990D881C02D4C815D816E817F819F2DF0
:106B6000C416D506E606970B97FFF1CF1196DC9376
:106B7000CE93B183A0831FBFDF91CF911F91FF9070
:106B8000EF90DF90CF90BF90AF9008955D010E948D
:106B90005A262F2DC616D706E806290B27FD25C035
:106BA00082E0CA30D80741F1F501D183C083C09299
:106BB0000E02D0920F02E0921002F0921102B092F7
:106BC0000B02A0920A028AE092E090932302809343
:106BD00022028091840090918500C2969093890052
:106BE0008093880082E086BBC6CF80912702811106
:106BF000D7CF83E00E94EB3780910A0290910B027D
:106C0000F50191838083D3CFCF93DF93CDB7DEB7E8
:106C100029970FB6F894DEBF0FBECDBF87E993E08A
:106C200090933B0280933A02FFB6F8941092800052
:106C300001E000938100E4E8F0E01182108280819D
:106C40009181C296909389008093880012E016BBD0
:106C500080819181C29690938B0080938A0084E01A
:106C600086BB80E092E00E94863506BB10936F00E1
:106C7000FFBE9DE088E10FB6F894A8958093600070
:106C80000FBE9093600080E4809360001093C0007A
:106C900087E090E09093C5008093C40086E08093E5
:106CA000C20088EB8093C10087E191E19F938F93AD
:106CB0000E94C0310F900F90F89483E592E00E94FB
:106CC000413A8C01892B19F478940E94C508F894F4
:106CD0000E945A26F62EE72ED82EC92EE2E2F2E0C6
:106CE0008581811101C0068382E292E022E0DC010D
:106CF00015962C9315970AE012E00D931C93EAE188
:106D0000F2E04481558166817781D80114964D93D4
:106D10005D936D937C931797DC011396FC93EE9330
:106D20001297D801ED93FC9382E192E091838083E6
:106D30008091840090918500C29690938900809301
:106D4000880026BB109252020E94D8288FEF8987B4
:106D500081E1B82E13C0F80143A14071648975899F
:106D600086890E94E918D80193968C91982F90718A
:106D700084FD9B2DF80193A310A2178E6CE873E19C
:106D8000CE0109960E945D118C01892B21F78FEFAE
:106D9000888709C0DC0195961C921E92949760E04A
:106DA00088960E946D2A68E87CE2CE0108960E94CF
:106DB0005D11009779F78FEF8F8302C00E94E9235E
:106DC00069E373E2CE0107960E945D110097B1F767
:106DD0008FEF8E831FEF0AC090910902828D981366
:106DE00002C010930902868D8111D1C06BE774E354
:106DF000CE0106960E945D11FC01892B69F78FEF89
:106E00008D8311E004C0FC01258120FDDAC065EA14
:106E100073E3CE0105960E945D110097A1F78FEFF5
:106E20008D830CC09C012D5F3F4FDC0112964C916D
:106E3000129760E08D919C910E9469196CE379E151
:106E4000CE0105960E945D11009761F78FEF8C834C
:106E500002E710E20BC02FB7F894992711969C9384
:106E60008E932FBF13830283128A118A6CEF74E111
:106E7000CE0104960E945D11FC01892B49F08785A3
:106E80009089A085B1852285222329F38C93EACFAE
:106E90008FEF8B830FC0F80164857585868540E090
:106EA0000E94E918D8011F966D917D918C9140E068
:106EB0000E94E91866EA7FE2CE0103960E945D1106
:106EC0008C01892B41F78FEF8A832FC0F8016185F0
:106ED0007285838540E00E94E918D8011C966D9167
:106EE0007D918C9140E00E94E918F80167857089D6
:106EF000818940E00E94E918D80152966D917D91F8
:106F00008C9140E00E94E918F801658976898789AB
:106F100040E00E94E918D80158966D917D918C91BE
:106F200040E00E94E918F80110866EE27CE1CE0193
:106F300002960E945D118C01892B41F68FEF8983A7
:106F400002C00E945D1F64EC7EE1CE0101960E94AA
:106F50005D110097B1F780E092E00E948635E2E291
:106F6000F2E081E08583789486811F928F93CF929F
:106F7000DF92EF92FF928DE091E19F938F930E94B9
:106F8000C0310FB6F894DEBF0FBECDBF9DCE8F5F70
:106F9000858F408951896289738980859185A28511
:106FA000B385840F951FA61FB71F808B918BA28B73
:106FB000B38B84839583A683B783CF010E948635E4
:106FC00015CF23FB442740F94127628173818481D7
:106FD0000E94E9181CCFF894682F70E083E592E0D6
:106FE0000E94633AFC0192899460928B109226026F
:106FF00081E08093510280E008957F928F929F926A
:10700000AF92BF92CF92DF92EF92FF920F931F93B6
:10701000CF93DF937C01DC01DC9162EA71E18D2F7B
:107020000E94C0288C01F701C481B084A184DC01D6
:1070300051969C90B2E09B1609F44FC00E945A26CC
:107040006B017C012B2D3A2D4C2F61E0D8011C9651
:107050008D919C911D970E9469190E945A268B015F
:107060009C010C191D092E093F090132134021050D
:10707000310558F54C2F50E0E1E09E1659F1AF92E2
:10708000BF925F934F93FF92EF92DF92CF921F9246
:10709000DF9388EB90E19F938F930E94C0318DB76F
:1070A0009EB70C960FB6F8949EBF0FBE8DBFDF91B2
:1070B000CF911F910F91FF90EF90DF90CF90BF90F5
:1070C000AF909F908F907F90089540E050E0E1E076
:1070D0009E12D5CF6B017C01D2CFDC011C96ED91C5
:1070E000FC911D9794808280738040E0682D772DFD
:1070F000892D0E94E9180E945A266B017C01B0E19B
:10710000CB0ED11CE11CF11C0E945A262F2DC61655
:10711000D706E806290B27FFF7CFF89441E0682D42
:10712000772D892D0E94E9180E945A266B017C0157
:1071300078942B2D3A2D4C2F61E0F80184859585AC
:107140000E9469194C2F50E09ACF0F931F93CF9351
:10715000DF9300D0CDB7DEB722E72B83DC011C968E
:10716000ED91FC911D978E010F5F1F4F22E0AE0144
:107170004D5F5F4F61E080810E94DB1789818F71D5
:1071800090E0982F88272A81822B0F900F900F90E4
:10719000DF91CF911F910F910895CF93DF93EC0171
:1071A00045969F938F938A891F928F938F858F9394
:1071B0008E858F931F926F938EEA90E19F938F93AA
:1071C0000E94C0311A8A8E859F8501969F878E877F
:1071D0008DB79EB70A960FB6F8949EBF0FBE8DBFAF
:1071E000DF91CF910895FF920F931F93CF93DF9379
:1071F0008C01FC01F08062EA71E18F2D0E94C028B1
:10720000EC010E943435188AF80180859185A285A9
:10721000B385892B8A2B8B2B01F58A89811118C0A4
:107220008F858F938E858F931F92FF9283EB90E1D2
:107230009F938F930E94C0310F900F900F900F90EB
:107240000F900F90DF91CF911F910F91FF900895B4
:107250006F2DCE010E94CD38E3CFF8018481958156
:10726000A681B7818C839D83AE83BF838085918502
:10727000A285B38588879987AA87BB871F861E86C4
:107280001A8A84858B8BCE01DF91CF911F910F914C
:10729000FF900C94863588E00E94EB37CF92DF9206
:1072A000EF92FF920F931F930E945A269F938F9302
:1072B0007F936F9301E010E020E030E0C0906F0218
:1072C000D0907002E0907102F09072026C157D0512
:1072D0008E059F0518F000E010E0980180916B0288
:1072E00090916C02A0916D02B0916E02800F911F7F
:1072F000A21FB31FBF93AF939F938F938EEF90E125
:107300009F938F930E94C0318DB79EB70A960FB698
:10731000F8949EBF0FBE8DBF1F910F91FF90EF900D
:10732000DF90CF9008950E945A269F938F937F936A
:107330006F9389EF90E19F938F930E94C0310F90DC
:107340000F900F900F900F900F900895F89498E081
:1073500088E10FB6F894A895809360000FBE9093D3
:107360006000FFCF1F920F920FB60F9211240BB641
:107370000F928F93EF93FF93E09196038091950383
:10738000E817A0F481E08E0F80939603F0E0EB5CA9
:10739000FC4F80818093C600FF91EF918F910F90F9
:1073A0000BBE0F900FBE0F901F9018958091C100DB
:1073B0008F7D8093C100F0CF1F920F920FB60F9276
:1073C00011240BB60F928F939F93EF93FF938091AD
:1073D000C6008E37B9F0E0913403E03C40F491E010
:1073E0009E0F90933403F0E0EC58FD4F8083FF91A3
:1073F000EF919F918F910F900BBE0F900FBE0F904A
:107400001F90189510922602E6CF1F920F920FB68A
:107410000F92112481E08093730285E30E94EB3781
:10742000DB018F939F930E94363ABF91AF91A29F49
:10743000800D911DA39F900DB29F900D1124089572
:107440006927962769277827872778270895A29F95
:10745000B001B39FC001A39F700D811D1124911D28
:10746000B29F700D811D1124911D08950E94273A2D
:10747000A59F900DB49F900DA49F800D911D112488
:107480000895DC012D923D924D925D926D927D9218
:107490008D929D92AD92BD92CD92DD92ED92FD9234
:1074A0000D931D93CD93DD930F90FF91EF918DB7C9
:1074B0008D938EB78D938FB78D93ED93FD93882722
:1074C00099270D9221C0DC01CB0181309105811DEE
:1074D0002D903D904D905D906D907D908D909D9004
:1074E000AD90BD90CD90DD90ED90FD900D911D91F2
:1074F000CD91DD91ED91FD910D90F894FEBF0FBE01
:10750000EDBFED91FD910D90EF93FF930F920895D4
:10751000FB01DC0102C005900D9241505040D8F7AC
:107520000895FC014150504030F001900616D1F70B
:107530003197CF010895882799270895FB01DC0131
:1075400002C001900D9241505040D8F7089568173D
:10755000790768F4FB01DC01E40FF51FA40FB51FE8
:1075600002C002900E9241505040D8F708950C94FA
:107570009E3ADC0101C06D9341505040E0F7089500
:04758000F894FFCFAD
:1075840000003A240080000010FF000011350000C4
:1075940000000000313500000080120213350000A5
:0A75A40000001A021A0200000000A5
:00000001FF
